Archive member included because of file (symbol)

c:/ti/ccsv5/tools/compiler/gcc-arm-none-eabi-4_7-2012q4/bin/../lib/gcc/arm-none-eabi/4.7.3/../../../../arm-none-eabi/lib\libc.a(lib_a-__atexit.o)
                              c:/ti/ccsv5/tools/compiler/gcc-arm-none-eabi-4_7-2012q4/bin/../lib/gcc/arm-none-eabi/4.7.3/../../../../arm-none-eabi/lib/rdimon-crt0.o (__register_exitproc)
c:/ti/ccsv5/tools/compiler/gcc-arm-none-eabi-4_7-2012q4/bin/../lib/gcc/arm-none-eabi/4.7.3/../../../../arm-none-eabi/lib\libc.a(lib_a-exit.o)
                              c:/ti/ccsv5/tools/compiler/gcc-arm-none-eabi-4_7-2012q4/bin/../lib/gcc/arm-none-eabi/4.7.3/../../../../arm-none-eabi/lib/rdimon-crt0.o (exit)
c:/ti/ccsv5/tools/compiler/gcc-arm-none-eabi-4_7-2012q4/bin/../lib/gcc/arm-none-eabi/4.7.3/../../../../arm-none-eabi/lib\libc.a(lib_a-fini.o)
                              c:/ti/ccsv5/tools/compiler/gcc-arm-none-eabi-4_7-2012q4/bin/../lib/gcc/arm-none-eabi/4.7.3/../../../../arm-none-eabi/lib/rdimon-crt0.o (__libc_fini_array)
c:/ti/ccsv5/tools/compiler/gcc-arm-none-eabi-4_7-2012q4/bin/../lib/gcc/arm-none-eabi/4.7.3/../../../../arm-none-eabi/lib\libc.a(lib_a-impure.o)
                              c:/ti/ccsv5/tools/compiler/gcc-arm-none-eabi-4_7-2012q4/bin/../lib/gcc/arm-none-eabi/4.7.3/../../../../arm-none-eabi/lib\libc.a(lib_a-__atexit.o) (_global_impure_ptr)
c:/ti/ccsv5/tools/compiler/gcc-arm-none-eabi-4_7-2012q4/bin/../lib/gcc/arm-none-eabi/4.7.3/../../../../arm-none-eabi/lib\libc.a(lib_a-init.o)
                              c:/ti/ccsv5/tools/compiler/gcc-arm-none-eabi-4_7-2012q4/bin/../lib/gcc/arm-none-eabi/4.7.3/../../../../arm-none-eabi/lib/rdimon-crt0.o (__libc_init_array)
c:/ti/ccsv5/tools/compiler/gcc-arm-none-eabi-4_7-2012q4/bin/../lib/gcc/arm-none-eabi/4.7.3/../../../../arm-none-eabi/lib\libc.a(lib_a-memset.o)
                              c:/ti/ccsv5/tools/compiler/gcc-arm-none-eabi-4_7-2012q4/bin/../lib/gcc/arm-none-eabi/4.7.3/../../../../arm-none-eabi/lib/rdimon-crt0.o (memset)
c:/ti/ccsv5/tools/compiler/gcc-arm-none-eabi-4_7-2012q4/bin/../lib/gcc/arm-none-eabi/4.7.3/../../../../arm-none-eabi/lib\libc.a(lib_a-printf.o)
                              ./main.o (printf)
c:/ti/ccsv5/tools/compiler/gcc-arm-none-eabi-4_7-2012q4/bin/../lib/gcc/arm-none-eabi/4.7.3/../../../../arm-none-eabi/lib\libc.a(lib_a-puts.o)
                              ./main.o (puts)
c:/ti/ccsv5/tools/compiler/gcc-arm-none-eabi-4_7-2012q4/bin/../lib/gcc/arm-none-eabi/4.7.3/../../../../arm-none-eabi/lib\libc.a(lib_a-strlen.o)
                              c:/ti/ccsv5/tools/compiler/gcc-arm-none-eabi-4_7-2012q4/bin/../lib/gcc/arm-none-eabi/4.7.3/../../../../arm-none-eabi/lib\libc.a(lib_a-puts.o) (strlen)
c:/ti/ccsv5/tools/compiler/gcc-arm-none-eabi-4_7-2012q4/bin/../lib/gcc/arm-none-eabi/4.7.3/../../../../arm-none-eabi/lib\libc.a(lib_a-vfprintf.o)
                              c:/ti/ccsv5/tools/compiler/gcc-arm-none-eabi-4_7-2012q4/bin/../lib/gcc/arm-none-eabi/4.7.3/../../../../arm-none-eabi/lib\libc.a(lib_a-printf.o) (_vfprintf_r)
c:/ti/ccsv5/tools/compiler/gcc-arm-none-eabi-4_7-2012q4/bin/../lib/gcc/arm-none-eabi/4.7.3/../../../../arm-none-eabi/lib\libc.a(lib_a-wsetup.o)
                              c:/ti/ccsv5/tools/compiler/gcc-arm-none-eabi-4_7-2012q4/bin/../lib/gcc/arm-none-eabi/4.7.3/../../../../arm-none-eabi/lib\libc.a(lib_a-vfprintf.o) (__swsetup_r)
c:/ti/ccsv5/tools/compiler/gcc-arm-none-eabi-4_7-2012q4/bin/../lib/gcc/arm-none-eabi/4.7.3/../../../../arm-none-eabi/lib\libc.a(lib_a-__call_atexit.o)
                              c:/ti/ccsv5/tools/compiler/gcc-arm-none-eabi-4_7-2012q4/bin/../lib/gcc/arm-none-eabi/4.7.3/../../../../arm-none-eabi/lib\libc.a(lib_a-exit.o) (__call_exitprocs)
c:/ti/ccsv5/tools/compiler/gcc-arm-none-eabi-4_7-2012q4/bin/../lib/gcc/arm-none-eabi/4.7.3/../../../../arm-none-eabi/lib\libc.a(lib_a-atexit.o)
                              c:/ti/ccsv5/tools/compiler/gcc-arm-none-eabi-4_7-2012q4/bin/../lib/gcc/arm-none-eabi/4.7.3/../../../../arm-none-eabi/lib\libc.a(lib_a-__call_atexit.o) (atexit)
c:/ti/ccsv5/tools/compiler/gcc-arm-none-eabi-4_7-2012q4/bin/../lib/gcc/arm-none-eabi/4.7.3/../../../../arm-none-eabi/lib\libc.a(lib_a-dtoa.o)
                              c:/ti/ccsv5/tools/compiler/gcc-arm-none-eabi-4_7-2012q4/bin/../lib/gcc/arm-none-eabi/4.7.3/../../../../arm-none-eabi/lib\libc.a(lib_a-vfprintf.o) (_dtoa_r)
c:/ti/ccsv5/tools/compiler/gcc-arm-none-eabi-4_7-2012q4/bin/../lib/gcc/arm-none-eabi/4.7.3/../../../../arm-none-eabi/lib\libc.a(lib_a-fflush.o)
                              c:/ti/ccsv5/tools/compiler/gcc-arm-none-eabi-4_7-2012q4/bin/../lib/gcc/arm-none-eabi/4.7.3/../../../../arm-none-eabi/lib\libc.a(lib_a-vfprintf.o) (_fflush_r)
c:/ti/ccsv5/tools/compiler/gcc-arm-none-eabi-4_7-2012q4/bin/../lib/gcc/arm-none-eabi/4.7.3/../../../../arm-none-eabi/lib\libc.a(lib_a-findfp.o)
                              c:/ti/ccsv5/tools/compiler/gcc-arm-none-eabi-4_7-2012q4/bin/../lib/gcc/arm-none-eabi/4.7.3/../../../../arm-none-eabi/lib\libc.a(lib_a-vfprintf.o) (__sinit)
c:/ti/ccsv5/tools/compiler/gcc-arm-none-eabi-4_7-2012q4/bin/../lib/gcc/arm-none-eabi/4.7.3/../../../../arm-none-eabi/lib\libc.a(lib_a-freer.o)
                              c:/ti/ccsv5/tools/compiler/gcc-arm-none-eabi-4_7-2012q4/bin/../lib/gcc/arm-none-eabi/4.7.3/../../../../arm-none-eabi/lib\libc.a(lib_a-wsetup.o) (_free_r)
c:/ti/ccsv5/tools/compiler/gcc-arm-none-eabi-4_7-2012q4/bin/../lib/gcc/arm-none-eabi/4.7.3/../../../../arm-none-eabi/lib\libc.a(lib_a-fvwrite.o)
                              c:/ti/ccsv5/tools/compiler/gcc-arm-none-eabi-4_7-2012q4/bin/../lib/gcc/arm-none-eabi/4.7.3/../../../../arm-none-eabi/lib\libc.a(lib_a-puts.o) (__sfvwrite_r)
c:/ti/ccsv5/tools/compiler/gcc-arm-none-eabi-4_7-2012q4/bin/../lib/gcc/arm-none-eabi/4.7.3/../../../../arm-none-eabi/lib\libc.a(lib_a-fwalk.o)
                              c:/ti/ccsv5/tools/compiler/gcc-arm-none-eabi-4_7-2012q4/bin/../lib/gcc/arm-none-eabi/4.7.3/../../../../arm-none-eabi/lib\libc.a(lib_a-findfp.o) (_fwalk)
c:/ti/ccsv5/tools/compiler/gcc-arm-none-eabi-4_7-2012q4/bin/../lib/gcc/arm-none-eabi/4.7.3/../../../../arm-none-eabi/lib\libc.a(lib_a-locale.o)
                              c:/ti/ccsv5/tools/compiler/gcc-arm-none-eabi-4_7-2012q4/bin/../lib/gcc/arm-none-eabi/4.7.3/../../../../arm-none-eabi/lib\libc.a(lib_a-vfprintf.o) (_localeconv_r)
c:/ti/ccsv5/tools/compiler/gcc-arm-none-eabi-4_7-2012q4/bin/../lib/gcc/arm-none-eabi/4.7.3/../../../../arm-none-eabi/lib\libc.a(lib_a-makebuf.o)
                              c:/ti/ccsv5/tools/compiler/gcc-arm-none-eabi-4_7-2012q4/bin/../lib/gcc/arm-none-eabi/4.7.3/../../../../arm-none-eabi/lib\libc.a(lib_a-wsetup.o) (__smakebuf_r)
c:/ti/ccsv5/tools/compiler/gcc-arm-none-eabi-4_7-2012q4/bin/../lib/gcc/arm-none-eabi/4.7.3/../../../../arm-none-eabi/lib\libc.a(lib_a-mallocr.o)
                              c:/ti/ccsv5/tools/compiler/gcc-arm-none-eabi-4_7-2012q4/bin/../lib/gcc/arm-none-eabi/4.7.3/../../../../arm-none-eabi/lib\libc.a(lib_a-findfp.o) (_malloc_r)
c:/ti/ccsv5/tools/compiler/gcc-arm-none-eabi-4_7-2012q4/bin/../lib/gcc/arm-none-eabi/4.7.3/../../../../arm-none-eabi/lib\libc.a(lib_a-memchr.o)
                              c:/ti/ccsv5/tools/compiler/gcc-arm-none-eabi-4_7-2012q4/bin/../lib/gcc/arm-none-eabi/4.7.3/../../../../arm-none-eabi/lib\libc.a(lib_a-vfprintf.o) (memchr)
c:/ti/ccsv5/tools/compiler/gcc-arm-none-eabi-4_7-2012q4/bin/../lib/gcc/arm-none-eabi/4.7.3/../../../../arm-none-eabi/lib\libc.a(lib_a-memcpy.o)
                              c:/ti/ccsv5/tools/compiler/gcc-arm-none-eabi-4_7-2012q4/bin/../lib/gcc/arm-none-eabi/4.7.3/../../../../arm-none-eabi/lib\libc.a(lib_a-dtoa.o) (memcpy)
c:/ti/ccsv5/tools/compiler/gcc-arm-none-eabi-4_7-2012q4/bin/../lib/gcc/arm-none-eabi/4.7.3/../../../../arm-none-eabi/lib\libc.a(lib_a-memmove.o)
                              c:/ti/ccsv5/tools/compiler/gcc-arm-none-eabi-4_7-2012q4/bin/../lib/gcc/arm-none-eabi/4.7.3/../../../../arm-none-eabi/lib\libc.a(lib_a-fvwrite.o) (memmove)
c:/ti/ccsv5/tools/compiler/gcc-arm-none-eabi-4_7-2012q4/bin/../lib/gcc/arm-none-eabi/4.7.3/../../../../arm-none-eabi/lib\libc.a(lib_a-mlock.o)
                              c:/ti/ccsv5/tools/compiler/gcc-arm-none-eabi-4_7-2012q4/bin/../lib/gcc/arm-none-eabi/4.7.3/../../../../arm-none-eabi/lib\libc.a(lib_a-freer.o) (__malloc_lock)
c:/ti/ccsv5/tools/compiler/gcc-arm-none-eabi-4_7-2012q4/bin/../lib/gcc/arm-none-eabi/4.7.3/../../../../arm-none-eabi/lib\libc.a(lib_a-mprec.o)
                              c:/ti/ccsv5/tools/compiler/gcc-arm-none-eabi-4_7-2012q4/bin/../lib/gcc/arm-none-eabi/4.7.3/../../../../arm-none-eabi/lib\libc.a(lib_a-dtoa.o) (_Balloc)
c:/ti/ccsv5/tools/compiler/gcc-arm-none-eabi-4_7-2012q4/bin/../lib/gcc/arm-none-eabi/4.7.3/../../../../arm-none-eabi/lib\libc.a(lib_a-reallocr.o)
                              c:/ti/ccsv5/tools/compiler/gcc-arm-none-eabi-4_7-2012q4/bin/../lib/gcc/arm-none-eabi/4.7.3/../../../../arm-none-eabi/lib\libc.a(lib_a-fvwrite.o) (_realloc_r)
c:/ti/ccsv5/tools/compiler/gcc-arm-none-eabi-4_7-2012q4/bin/../lib/gcc/arm-none-eabi/4.7.3/../../../../arm-none-eabi/lib\libc.a(lib_a-s_fpclassify.o)
                              c:/ti/ccsv5/tools/compiler/gcc-arm-none-eabi-4_7-2012q4/bin/../lib/gcc/arm-none-eabi/4.7.3/../../../../arm-none-eabi/lib\libc.a(lib_a-vfprintf.o) (__fpclassifyd)
c:/ti/ccsv5/tools/compiler/gcc-arm-none-eabi-4_7-2012q4/bin/../lib/gcc/arm-none-eabi/4.7.3/../../../../arm-none-eabi/lib\libc.a(lib_a-sbrkr.o)
                              c:/ti/ccsv5/tools/compiler/gcc-arm-none-eabi-4_7-2012q4/bin/../lib/gcc/arm-none-eabi/4.7.3/../../../../arm-none-eabi/lib\libc.a(lib_a-freer.o) (_sbrk_r)
c:/ti/ccsv5/tools/compiler/gcc-arm-none-eabi-4_7-2012q4/bin/../lib/gcc/arm-none-eabi/4.7.3/../../../../arm-none-eabi/lib\libc.a(lib_a-stdio.o)
                              c:/ti/ccsv5/tools/compiler/gcc-arm-none-eabi-4_7-2012q4/bin/../lib/gcc/arm-none-eabi/4.7.3/../../../../arm-none-eabi/lib\libc.a(lib_a-findfp.o) (__sread)
c:/ti/ccsv5/tools/compiler/gcc-arm-none-eabi-4_7-2012q4/bin/../lib/gcc/arm-none-eabi/4.7.3/../../../../arm-none-eabi/lib\libc.a(lib_a-strcmp.o)
                              c:/ti/ccsv5/tools/compiler/gcc-arm-none-eabi-4_7-2012q4/bin/../lib/gcc/arm-none-eabi/4.7.3/../../../../arm-none-eabi/lib\libc.a(lib_a-locale.o) (strcmp)
c:/ti/ccsv5/tools/compiler/gcc-arm-none-eabi-4_7-2012q4/bin/../lib/gcc/arm-none-eabi/4.7.3/../../../../arm-none-eabi/lib\libc.a(lib_a-vfiprintf.o)
                              c:/ti/ccsv5/tools/compiler/gcc-arm-none-eabi-4_7-2012q4/bin/../lib/gcc/arm-none-eabi/4.7.3/../../../../arm-none-eabi/lib\libc.a(lib_a-vfprintf.o) (__sprint_r)
c:/ti/ccsv5/tools/compiler/gcc-arm-none-eabi-4_7-2012q4/bin/../lib/gcc/arm-none-eabi/4.7.3/../../../../arm-none-eabi/lib\libc.a(lib_a-writer.o)
                              c:/ti/ccsv5/tools/compiler/gcc-arm-none-eabi-4_7-2012q4/bin/../lib/gcc/arm-none-eabi/4.7.3/../../../../arm-none-eabi/lib\libc.a(lib_a-stdio.o) (_write_r)
c:/ti/ccsv5/tools/compiler/gcc-arm-none-eabi-4_7-2012q4/bin/../lib/gcc/arm-none-eabi/4.7.3/../../../../arm-none-eabi/lib\libc.a(lib_a-callocr.o)
                              c:/ti/ccsv5/tools/compiler/gcc-arm-none-eabi-4_7-2012q4/bin/../lib/gcc/arm-none-eabi/4.7.3/../../../../arm-none-eabi/lib\libc.a(lib_a-mprec.o) (_calloc_r)
c:/ti/ccsv5/tools/compiler/gcc-arm-none-eabi-4_7-2012q4/bin/../lib/gcc/arm-none-eabi/4.7.3/../../../../arm-none-eabi/lib\libc.a(lib_a-closer.o)
                              c:/ti/ccsv5/tools/compiler/gcc-arm-none-eabi-4_7-2012q4/bin/../lib/gcc/arm-none-eabi/4.7.3/../../../../arm-none-eabi/lib\libc.a(lib_a-stdio.o) (_close_r)
c:/ti/ccsv5/tools/compiler/gcc-arm-none-eabi-4_7-2012q4/bin/../lib/gcc/arm-none-eabi/4.7.3/../../../../arm-none-eabi/lib\libc.a(lib_a-fclose.o)
                              c:/ti/ccsv5/tools/compiler/gcc-arm-none-eabi-4_7-2012q4/bin/../lib/gcc/arm-none-eabi/4.7.3/../../../../arm-none-eabi/lib\libc.a(lib_a-findfp.o) (fclose)
c:/ti/ccsv5/tools/compiler/gcc-arm-none-eabi-4_7-2012q4/bin/../lib/gcc/arm-none-eabi/4.7.3/../../../../arm-none-eabi/lib\libc.a(lib_a-fputwc.o)
                              c:/ti/ccsv5/tools/compiler/gcc-arm-none-eabi-4_7-2012q4/bin/../lib/gcc/arm-none-eabi/4.7.3/../../../../arm-none-eabi/lib\libc.a(lib_a-vfiprintf.o) (_fputwc_r)
c:/ti/ccsv5/tools/compiler/gcc-arm-none-eabi-4_7-2012q4/bin/../lib/gcc/arm-none-eabi/4.7.3/../../../../arm-none-eabi/lib\libc.a(lib_a-fstatr.o)
                              c:/ti/ccsv5/tools/compiler/gcc-arm-none-eabi-4_7-2012q4/bin/../lib/gcc/arm-none-eabi/4.7.3/../../../../arm-none-eabi/lib\libc.a(lib_a-makebuf.o) (_fstat_r)
c:/ti/ccsv5/tools/compiler/gcc-arm-none-eabi-4_7-2012q4/bin/../lib/gcc/arm-none-eabi/4.7.3/../../../../arm-none-eabi/lib\libc.a(lib_a-isattyr.o)
                              c:/ti/ccsv5/tools/compiler/gcc-arm-none-eabi-4_7-2012q4/bin/../lib/gcc/arm-none-eabi/4.7.3/../../../../arm-none-eabi/lib\libc.a(lib_a-makebuf.o) (_isatty_r)
c:/ti/ccsv5/tools/compiler/gcc-arm-none-eabi-4_7-2012q4/bin/../lib/gcc/arm-none-eabi/4.7.3/../../../../arm-none-eabi/lib\libc.a(lib_a-lseekr.o)
                              c:/ti/ccsv5/tools/compiler/gcc-arm-none-eabi-4_7-2012q4/bin/../lib/gcc/arm-none-eabi/4.7.3/../../../../arm-none-eabi/lib\libc.a(lib_a-stdio.o) (_lseek_r)
c:/ti/ccsv5/tools/compiler/gcc-arm-none-eabi-4_7-2012q4/bin/../lib/gcc/arm-none-eabi/4.7.3/../../../../arm-none-eabi/lib\libc.a(lib_a-readr.o)
                              c:/ti/ccsv5/tools/compiler/gcc-arm-none-eabi-4_7-2012q4/bin/../lib/gcc/arm-none-eabi/4.7.3/../../../../arm-none-eabi/lib\libc.a(lib_a-stdio.o) (_read_r)
c:/ti/ccsv5/tools/compiler/gcc-arm-none-eabi-4_7-2012q4/bin/../lib/gcc/arm-none-eabi/4.7.3/../../../../arm-none-eabi/lib\libc.a(lib_a-reent.o)
                              c:/ti/ccsv5/tools/compiler/gcc-arm-none-eabi-4_7-2012q4/bin/../lib/gcc/arm-none-eabi/4.7.3/../../../../arm-none-eabi/lib\libc.a(lib_a-sbrkr.o) (errno)
c:/ti/ccsv5/tools/compiler/gcc-arm-none-eabi-4_7-2012q4/bin/../lib/gcc/arm-none-eabi/4.7.3/../../../../arm-none-eabi/lib\libc.a(lib_a-wbuf.o)
                              c:/ti/ccsv5/tools/compiler/gcc-arm-none-eabi-4_7-2012q4/bin/../lib/gcc/arm-none-eabi/4.7.3/../../../../arm-none-eabi/lib\libc.a(lib_a-fputwc.o) (__swbuf_r)
c:/ti/ccsv5/tools/compiler/gcc-arm-none-eabi-4_7-2012q4/bin/../lib/gcc/arm-none-eabi/4.7.3/../../../../arm-none-eabi/lib\libc.a(lib_a-wcrtomb.o)
                              c:/ti/ccsv5/tools/compiler/gcc-arm-none-eabi-4_7-2012q4/bin/../lib/gcc/arm-none-eabi/4.7.3/../../../../arm-none-eabi/lib\libc.a(lib_a-fputwc.o) (_wcrtomb_r)
c:/ti/ccsv5/tools/compiler/gcc-arm-none-eabi-4_7-2012q4/bin/../lib/gcc/arm-none-eabi/4.7.3/../../../../arm-none-eabi/lib\libc.a(lib_a-wctomb_r.o)
                              c:/ti/ccsv5/tools/compiler/gcc-arm-none-eabi-4_7-2012q4/bin/../lib/gcc/arm-none-eabi/4.7.3/../../../../arm-none-eabi/lib\libc.a(lib_a-wcrtomb.o) (__wctomb)
c:/ti/ccsv5/tools/compiler/gcc-arm-none-eabi-4_7-2012q4/bin/../lib/gcc/arm-none-eabi/4.7.3\libgcc.a(_udivsi3.o)
                              c:/ti/ccsv5/tools/compiler/gcc-arm-none-eabi-4_7-2012q4/bin/../lib/gcc/arm-none-eabi/4.7.3/../../../../arm-none-eabi/lib\libc.a(lib_a-dtoa.o) (__aeabi_uidiv)
c:/ti/ccsv5/tools/compiler/gcc-arm-none-eabi-4_7-2012q4/bin/../lib/gcc/arm-none-eabi/4.7.3\libgcc.a(_dvmd_tls.o)
                              c:/ti/ccsv5/tools/compiler/gcc-arm-none-eabi-4_7-2012q4/bin/../lib/gcc/arm-none-eabi/4.7.3\libgcc.a(_udivsi3.o) (__aeabi_idiv0)
c:/ti/ccsv5/tools/compiler/gcc-arm-none-eabi-4_7-2012q4/bin/../lib/gcc/arm-none-eabi/4.7.3\libgcc.a(_arm_addsubdf3.o)
                              c:/ti/ccsv5/tools/compiler/gcc-arm-none-eabi-4_7-2012q4/bin/../lib/gcc/arm-none-eabi/4.7.3/../../../../arm-none-eabi/lib\libc.a(lib_a-dtoa.o) (__aeabi_dsub)
c:/ti/ccsv5/tools/compiler/gcc-arm-none-eabi-4_7-2012q4/bin/../lib/gcc/arm-none-eabi/4.7.3\libgcc.a(_arm_muldivdf3.o)
                              c:/ti/ccsv5/tools/compiler/gcc-arm-none-eabi-4_7-2012q4/bin/../lib/gcc/arm-none-eabi/4.7.3/../../../../arm-none-eabi/lib\libc.a(lib_a-dtoa.o) (__aeabi_dmul)
c:/ti/ccsv5/tools/compiler/gcc-arm-none-eabi-4_7-2012q4/bin/../lib/gcc/arm-none-eabi/4.7.3\libgcc.a(_arm_cmpdf2.o)
                              c:/ti/ccsv5/tools/compiler/gcc-arm-none-eabi-4_7-2012q4/bin/../lib/gcc/arm-none-eabi/4.7.3/../../../../arm-none-eabi/lib\libc.a(lib_a-vfprintf.o) (__aeabi_dcmpeq)
c:/ti/ccsv5/tools/compiler/gcc-arm-none-eabi-4_7-2012q4/bin/../lib/gcc/arm-none-eabi/4.7.3\libgcc.a(_arm_fixdfsi.o)
                              c:/ti/ccsv5/tools/compiler/gcc-arm-none-eabi-4_7-2012q4/bin/../lib/gcc/arm-none-eabi/4.7.3/../../../../arm-none-eabi/lib\libc.a(lib_a-dtoa.o) (__aeabi_d2iz)
c:/ti/ccsv5/tools/compiler/gcc-arm-none-eabi-4_7-2012q4/bin/../lib/gcc/arm-none-eabi/4.7.3\libgcc.a(_aeabi_uldivmod.o)
                              c:/ti/ccsv5/tools/compiler/gcc-arm-none-eabi-4_7-2012q4/bin/../lib/gcc/arm-none-eabi/4.7.3/../../../../arm-none-eabi/lib\libc.a(lib_a-vfprintf.o) (__aeabi_uldivmod)
c:/ti/ccsv5/tools/compiler/gcc-arm-none-eabi-4_7-2012q4/bin/../lib/gcc/arm-none-eabi/4.7.3\libgcc.a(bpabi.o)
                              c:/ti/ccsv5/tools/compiler/gcc-arm-none-eabi-4_7-2012q4/bin/../lib/gcc/arm-none-eabi/4.7.3\libgcc.a(_aeabi_uldivmod.o) (__gnu_uldivmod_helper)
c:/ti/ccsv5/tools/compiler/gcc-arm-none-eabi-4_7-2012q4/bin/../lib/gcc/arm-none-eabi/4.7.3\libgcc.a(_divdi3.o)
                              c:/ti/ccsv5/tools/compiler/gcc-arm-none-eabi-4_7-2012q4/bin/../lib/gcc/arm-none-eabi/4.7.3\libgcc.a(bpabi.o) (__divdi3)
c:/ti/ccsv5/tools/compiler/gcc-arm-none-eabi-4_7-2012q4/bin/../lib/gcc/arm-none-eabi/4.7.3\libgcc.a(_udivdi3.o)
                              c:/ti/ccsv5/tools/compiler/gcc-arm-none-eabi-4_7-2012q4/bin/../lib/gcc/arm-none-eabi/4.7.3\libgcc.a(bpabi.o) (__udivdi3)
c:/ti/ccsv5/tools/compiler/gcc-arm-none-eabi-4_7-2012q4/bin/../lib/gcc/arm-none-eabi/4.7.3\libgcc.a(_clzsi2.o)
                              c:/ti/ccsv5/tools/compiler/gcc-arm-none-eabi-4_7-2012q4/bin/../lib/gcc/arm-none-eabi/4.7.3\libgcc.a(_divdi3.o) (__clzsi2)
c:/ti/ccsv5/tools/compiler/gcc-arm-none-eabi-4_7-2012q4/bin/../lib/gcc/arm-none-eabi/4.7.3/../../../../arm-none-eabi/lib\librdimon.a(rdimon-syscalls.o)
                              c:/ti/ccsv5/tools/compiler/gcc-arm-none-eabi-4_7-2012q4/bin/../lib/gcc/arm-none-eabi/4.7.3/../../../../arm-none-eabi/lib/rdimon-crt0.o (initialise_monitor_handles)
c:/ti/ccsv5/tools/compiler/gcc-arm-none-eabi-4_7-2012q4/bin/../lib/gcc/arm-none-eabi/4.7.3/../../../../arm-none-eabi/lib\librdimon.a(rdimon-_exit.o)
                              c:/ti/ccsv5/tools/compiler/gcc-arm-none-eabi-4_7-2012q4/bin/../lib/gcc/arm-none-eabi/4.7.3/../../../../arm-none-eabi/lib\libc.a(lib_a-exit.o) (_exit)
c:/ti/ccsv5/tools/compiler/gcc-arm-none-eabi-4_7-2012q4/bin/../lib/gcc/arm-none-eabi/4.7.3/../../../../arm-none-eabi/lib\librdimon.a(rdimon-_kill.o)
                              c:/ti/ccsv5/tools/compiler/gcc-arm-none-eabi-4_7-2012q4/bin/../lib/gcc/arm-none-eabi/4.7.3/../../../../arm-none-eabi/lib\librdimon.a(rdimon-_exit.o) (_kill)
c:/ti/ccsv5/tools/compiler/gcc-arm-none-eabi-4_7-2012q4/bin/../lib/gcc/arm-none-eabi/4.7.3/../../../../arm-none-eabi/lib\libc.a(lib_a-errno.o)
                              c:/ti/ccsv5/tools/compiler/gcc-arm-none-eabi-4_7-2012q4/bin/../lib/gcc/arm-none-eabi/4.7.3/../../../../arm-none-eabi/lib\librdimon.a(rdimon-syscalls.o) (__errno)

Allocating common symbols
Common symbol       size              file

errno               0x4               c:/ti/ccsv5/tools/compiler/gcc-arm-none-eabi-4_7-2012q4/bin/../lib/gcc/arm-none-eabi/4.7.3/../../../../arm-none-eabi/lib\libc.a(lib_a-reent.o)

Memory Configuration

Name             Origin             Length             Attributes
SRAM             0x0c2f0400         0x0000fc00
L3OCMC0          0x0c300000         0x00010000
M3SHUMEM         0x0c310000         0x00004000
M3SHDMEM         0x0c350000         0x00002000
DDR0             0x80000000         0x40000000
*default*        0x00000000         0xffffffff

Linker script and memory map

LOAD c:/ti/ccsv5/tools/compiler/gcc-arm-none-eabi-4_7-2012q4/bin/../lib/gcc/arm-none-eabi/4.7.3/../../../../arm-none-eabi/lib\librdimon.a
LOAD c:/ti/ccsv5/tools/compiler/gcc-arm-none-eabi-4_7-2012q4/bin/../lib/gcc/arm-none-eabi/4.7.3/crti.o
LOAD c:/ti/ccsv5/tools/compiler/gcc-arm-none-eabi-4_7-2012q4/bin/../lib/gcc/arm-none-eabi/4.7.3/crtbegin.o
LOAD c:/ti/ccsv5/tools/compiler/gcc-arm-none-eabi-4_7-2012q4/bin/../lib/gcc/arm-none-eabi/4.7.3/../../../../arm-none-eabi/lib/rdimon-crt0.o
                0x00004000                HEAPSIZE = 0x4000
                0x00001000                STACKSIZE = 0x1000
LOAD ./common_arm/v7_pmu.o
LOAD ./common_arm/utilFxns.o
LOAD ./common_arm/arm_utility.o
LOAD ./common_arm/arm_cpintc.o
LOAD ./common_arm/aintc_inth.o
LOAD ./common_arm/GIC_ctl.o
LOAD ./common_arm/Cortex_A_generic_timer.o
LOAD ./startup_ARMCA8.o
LOAD ./main.o
START GROUP
LOAD c:/ti/ccsv5/tools/compiler/gcc-arm-none-eabi-4_7-2012q4/bin/../lib/gcc/arm-none-eabi/4.7.3/../../../../arm-none-eabi/lib\libc.a
LOAD c:/ti/ccsv5/tools/compiler/gcc-arm-none-eabi-4_7-2012q4/bin/../lib/gcc/arm-none-eabi/4.7.3\libgcc.a
LOAD c:/ti/ccsv5/tools/compiler/gcc-arm-none-eabi-4_7-2012q4/bin/../lib/gcc/arm-none-eabi/4.7.3/../../../../arm-none-eabi/lib\librdimon.a
END GROUP

.rsthand        0x80000000       0x90
                0x80000000                . = ALIGN (0x10000)
 *(.isr_vector)
 .isr_vector    0x80000000       0x70 ./startup_ARMCA8.o
                0x80000000                __isr_vector
                0x80000066                DEF_IRQHandler
 *startup_ARMCA8.o(.text)
 .text          0x80000070       0x20 ./startup_ARMCA8.o
                0x80000070                Entry
                0x80000090                . = ALIGN (0x4)

.text           0x80000090     0xc788
 *(.text*)
 .text          0x80000090        0x0 c:/ti/ccsv5/tools/compiler/gcc-arm-none-eabi-4_7-2012q4/bin/../lib/gcc/arm-none-eabi/4.7.3/crti.o
 .text          0x80000090       0x94 c:/ti/ccsv5/tools/compiler/gcc-arm-none-eabi-4_7-2012q4/bin/../lib/gcc/arm-none-eabi/4.7.3/crtbegin.o
 .text          0x80000124      0x12c c:/ti/ccsv5/tools/compiler/gcc-arm-none-eabi-4_7-2012q4/bin/../lib/gcc/arm-none-eabi/4.7.3/../../../../arm-none-eabi/lib/rdimon-crt0.o
                0x80000124                _start
                0x80000124                start
                0x80000124                _mainCRTStartup
 .text          0x80000250      0x154 ./common_arm/v7_pmu.o
                0x80000250                _getPMN
                0x80000260                _pmn_config
                0x80000274                _ccnt_divider
                0x8000028c                _enable_pmu
                0x8000029c                _disable_pmu
                0x800002ac                _enable_ccnt
                0x800002b8                _disable_ccnt
                0x800002c4                _enable_pmn
                0x800002d4                _disable_pmn
                0x800002e4                _enable_pmu_user_access
                0x800002f8                _disable_pmu_user_access
                0x8000030c                _read_ccnt
                0x80000314                _read_pmn
                0x80000328                _pmu_software_increment
                0x80000338                _read_flags
                0x80000340                _write_flags
                0x8000034c                _enable_ccnt_irq
                0x80000358                _disable_ccnt_irq
                0x80000364                _enable_pmn_irq
                0x80000374                _disable_pmn_irq
                0x80000384                _reset_pmn
                0x80000394                _reset_ccnt
 .text          0x800003a4        0x8 ./common_arm/utilFxns.o
                0x800003a4                regByteWrite
 .text          0x800003ac      0xacc ./common_arm/arm_utility.o
                0x800003ac                read_cpu_id
                0x800003b8                goto_user_mode
                0x800003dc                arm_enable_irq
                0x800003f4                svc_intr_isr
                0x80000414                arm_disable_cache
                0x80000428                arm_enable_cache
                0x80000440                arm_enable_mmu
                0x80000458                flush_tlb
                0x80000468                lpae_mmu_enable
                0x800004b0                cache_ctlr_setup
                0x800004e0                Set_MSMC_As_Sharable
                0x80000668                Level_2_lpae_setup
                0x80000990                Level_3_lpae_setup
                0x80000e68                DSB_inst
 .text          0x80000e78       0x98 ./common_arm/arm_cpintc.o
                0x80000e78                Arm_Cpintc_Init
                0x80000e98                Arm_Cpintc_MapSysToHostInt
                0x80000eb8                Arm_Cpintc_EnableChannel
                0x80000ed8                Arm_Cpintc_SetSysInterrupt
                0x80000ef4                Arm_Cpintc_ClearSysInterrupt
 .text          0x80000f10      0x2b4 ./common_arm/aintc_inth.o
                0x80000f10                INTH_InitHandler
                0x80000f64                INTH_RegisterHandler
                0x80000f84                INTH_SetupInterrupt
                0x80001038                INTH_EnableInterrupt
                0x8000105c                INTH_DisableInterrupt
                0x80001080                INTH_GetIntCount
                0x8000109c                INTH_GetIntHandler
                0x800010b8                INTH_SetSwInt
                0x800010e0                INTH_ClearIntCount
                0x800010fc                INTH_SetEndOfInt
                0x80001110                INTH_DeactivateInt
                0x80001124                INTH_Set_Pending
                0x80001138                INTH_Clear_Pending
                0x8000114c                INTH_Set_Active
                0x80001160                INTH_Clear_Active
                0x80001174                INTH_IRQHandler
 .text          0x800011c4      0x394 ./common_arm/GIC_ctl.o
                0x800011c4                GICD_Global_Enable_Disable
                0x80001254                GICD_Intr_Enable_Disable
                0x80001280                GICD_SetTriggerType
                0x800012cc                GICD_TriggerSGI
                0x80001308                GICD_Set_Pending
                0x80001340                GICD_Clear_Pending
                0x80001378                GICD_Set_Active
                0x80001398                GICD_Clear_Active
                0x800013b8                GICD_Set_Intr_Group
                0x800013e0                GICD_Set_Group1_Intr_Priority
                0x80001404                GICD_Set_Intr_Targets
                0x8000141c                GICD_InitDistributor
                0x80001484                GICC_InitCPUInterface
                0x800014a0                GICC_GetIntId
                0x800014c4                GICC_EndOfInt
                0x800014d0                GICC_DeactInt
                0x800014dc                GIC_Init
 .text          0x80001558       0x58 ./common_arm/Cortex_A_generic_timer.o
                0x80001558                GTimer_getCounterFrequency
                0x80001560                GTimer_getPhysicalCounter
                0x80001568                GTimer_getPL1PhyTmrCtrl
                0x80001570                GTimer_setPL1PhyTmrCtrl
                0x80001590                GTimer_getPL1PhyTmrTmrValue
                0x80001598                GTimer_setPL1PhyTmrTmrValue
                0x800015a0                GTimer_getPL1PhyTmrCmpValue
 .text          0x800015b0       0x84 ./main.o
                0x800015b0                Interrupt_ISR
                0x80001604                Interrupt_Init
 .text.startup  0x80001634       0x54 ./main.o
                0x80001634                main
 .text          0x80001688        0x0 c:/ti/ccsv5/tools/compiler/gcc-arm-none-eabi-4_7-2012q4/bin/../lib/gcc/arm-none-eabi/4.7.3/../../../../arm-none-eabi/lib\libc.a(lib_a-__atexit.o)
 .text.__register_exitproc
                0x80001688       0xf4 c:/ti/ccsv5/tools/compiler/gcc-arm-none-eabi-4_7-2012q4/bin/../lib/gcc/arm-none-eabi/4.7.3/../../../../arm-none-eabi/lib\libc.a(lib_a-__atexit.o)
                0x80001688                __register_exitproc
 .text          0x8000177c        0x0 c:/ti/ccsv5/tools/compiler/gcc-arm-none-eabi-4_7-2012q4/bin/../lib/gcc/arm-none-eabi/4.7.3/../../../../arm-none-eabi/lib\libc.a(lib_a-exit.o)
 .text.exit     0x8000177c       0x34 c:/ti/ccsv5/tools/compiler/gcc-arm-none-eabi-4_7-2012q4/bin/../lib/gcc/arm-none-eabi/4.7.3/../../../../arm-none-eabi/lib\libc.a(lib_a-exit.o)
                0x8000177c                exit
 .text          0x800017b0        0x0 c:/ti/ccsv5/tools/compiler/gcc-arm-none-eabi-4_7-2012q4/bin/../lib/gcc/arm-none-eabi/4.7.3/../../../../arm-none-eabi/lib\libc.a(lib_a-fini.o)
 .text.__libc_fini_array
                0x800017b0       0x44 c:/ti/ccsv5/tools/compiler/gcc-arm-none-eabi-4_7-2012q4/bin/../lib/gcc/arm-none-eabi/4.7.3/../../../../arm-none-eabi/lib\libc.a(lib_a-fini.o)
                0x800017b0                __libc_fini_array
 .text          0x800017f4        0x0 c:/ti/ccsv5/tools/compiler/gcc-arm-none-eabi-4_7-2012q4/bin/../lib/gcc/arm-none-eabi/4.7.3/../../../../arm-none-eabi/lib\libc.a(lib_a-impure.o)
 .text          0x800017f4        0x0 c:/ti/ccsv5/tools/compiler/gcc-arm-none-eabi-4_7-2012q4/bin/../lib/gcc/arm-none-eabi/4.7.3/../../../../arm-none-eabi/lib\libc.a(lib_a-init.o)
 .text.__libc_init_array
                0x800017f4       0x88 c:/ti/ccsv5/tools/compiler/gcc-arm-none-eabi-4_7-2012q4/bin/../lib/gcc/arm-none-eabi/4.7.3/../../../../arm-none-eabi/lib\libc.a(lib_a-init.o)
                0x800017f4                __libc_init_array
 .text          0x8000187c        0x0 c:/ti/ccsv5/tools/compiler/gcc-arm-none-eabi-4_7-2012q4/bin/../lib/gcc/arm-none-eabi/4.7.3/../../../../arm-none-eabi/lib\libc.a(lib_a-memset.o)
 .text.memset   0x8000187c       0xf8 c:/ti/ccsv5/tools/compiler/gcc-arm-none-eabi-4_7-2012q4/bin/../lib/gcc/arm-none-eabi/4.7.3/../../../../arm-none-eabi/lib\libc.a(lib_a-memset.o)
                0x8000187c                memset
 .text          0x80001974        0x0 c:/ti/ccsv5/tools/compiler/gcc-arm-none-eabi-4_7-2012q4/bin/../lib/gcc/arm-none-eabi/4.7.3/../../../../arm-none-eabi/lib\libc.a(lib_a-printf.o)
 .text._printf_r
                0x80001974       0x34 c:/ti/ccsv5/tools/compiler/gcc-arm-none-eabi-4_7-2012q4/bin/../lib/gcc/arm-none-eabi/4.7.3/../../../../arm-none-eabi/lib\libc.a(lib_a-printf.o)
                0x80001974                _printf_r
 .text.printf   0x800019a8       0x40 c:/ti/ccsv5/tools/compiler/gcc-arm-none-eabi-4_7-2012q4/bin/../lib/gcc/arm-none-eabi/4.7.3/../../../../arm-none-eabi/lib\libc.a(lib_a-printf.o)
                0x800019a8                printf
 .text          0x800019e8        0x0 c:/ti/ccsv5/tools/compiler/gcc-arm-none-eabi-4_7-2012q4/bin/../lib/gcc/arm-none-eabi/4.7.3/../../../../arm-none-eabi/lib\libc.a(lib_a-puts.o)
 .text._puts_r  0x800019e8       0xa4 c:/ti/ccsv5/tools/compiler/gcc-arm-none-eabi-4_7-2012q4/bin/../lib/gcc/arm-none-eabi/4.7.3/../../../../arm-none-eabi/lib\libc.a(lib_a-puts.o)
                0x800019e8                _puts_r
 .text.puts     0x80001a8c       0x14 c:/ti/ccsv5/tools/compiler/gcc-arm-none-eabi-4_7-2012q4/bin/../lib/gcc/arm-none-eabi/4.7.3/../../../../arm-none-eabi/lib\libc.a(lib_a-puts.o)
                0x80001a8c                puts
 .text          0x80001aa0        0x0 c:/ti/ccsv5/tools/compiler/gcc-arm-none-eabi-4_7-2012q4/bin/../lib/gcc/arm-none-eabi/4.7.3/../../../../arm-none-eabi/lib\libc.a(lib_a-strlen.o)
 .text.strlen   0x80001aa0       0x60 c:/ti/ccsv5/tools/compiler/gcc-arm-none-eabi-4_7-2012q4/bin/../lib/gcc/arm-none-eabi/4.7.3/../../../../arm-none-eabi/lib\libc.a(lib_a-strlen.o)
                0x80001aa0                strlen
 .text          0x80001b00        0x0 c:/ti/ccsv5/tools/compiler/gcc-arm-none-eabi-4_7-2012q4/bin/../lib/gcc/arm-none-eabi/4.7.3/../../../../arm-none-eabi/lib\libc.a(lib_a-vfprintf.o)
 .text._vfprintf_r
                0x80001b00     0x2158 c:/ti/ccsv5/tools/compiler/gcc-arm-none-eabi-4_7-2012q4/bin/../lib/gcc/arm-none-eabi/4.7.3/../../../../arm-none-eabi/lib\libc.a(lib_a-vfprintf.o)
                0x80001b00                _vfprintf_r
 .text.vfprintf
                0x80003c58       0x2c c:/ti/ccsv5/tools/compiler/gcc-arm-none-eabi-4_7-2012q4/bin/../lib/gcc/arm-none-eabi/4.7.3/../../../../arm-none-eabi/lib\libc.a(lib_a-vfprintf.o)
                0x80003c58                vfprintf
 .text          0x80003c84        0x0 c:/ti/ccsv5/tools/compiler/gcc-arm-none-eabi-4_7-2012q4/bin/../lib/gcc/arm-none-eabi/4.7.3/../../../../arm-none-eabi/lib\libc.a(lib_a-wsetup.o)
 .text.__swsetup_r
                0x80003c84      0x138 c:/ti/ccsv5/tools/compiler/gcc-arm-none-eabi-4_7-2012q4/bin/../lib/gcc/arm-none-eabi/4.7.3/../../../../arm-none-eabi/lib\libc.a(lib_a-wsetup.o)
                0x80003c84                __swsetup_r
 .text          0x80003dbc        0x0 c:/ti/ccsv5/tools/compiler/gcc-arm-none-eabi-4_7-2012q4/bin/../lib/gcc/arm-none-eabi/4.7.3/../../../../arm-none-eabi/lib\libc.a(lib_a-__call_atexit.o)
 .text.startup.register_fini
                0x80003dbc       0x24 c:/ti/ccsv5/tools/compiler/gcc-arm-none-eabi-4_7-2012q4/bin/../lib/gcc/arm-none-eabi/4.7.3/../../../../arm-none-eabi/lib\libc.a(lib_a-__call_atexit.o)
 .text.__call_exitprocs
                0x80003de0      0x17c c:/ti/ccsv5/tools/compiler/gcc-arm-none-eabi-4_7-2012q4/bin/../lib/gcc/arm-none-eabi/4.7.3/../../../../arm-none-eabi/lib\libc.a(lib_a-__call_atexit.o)
                0x80003de0                __call_exitprocs
 .text          0x80003f5c        0x0 c:/ti/ccsv5/tools/compiler/gcc-arm-none-eabi-4_7-2012q4/bin/../lib/gcc/arm-none-eabi/4.7.3/../../../../arm-none-eabi/lib\libc.a(lib_a-atexit.o)
 .text.atexit   0x80003f5c       0x20 c:/ti/ccsv5/tools/compiler/gcc-arm-none-eabi-4_7-2012q4/bin/../lib/gcc/arm-none-eabi/4.7.3/../../../../arm-none-eabi/lib\libc.a(lib_a-atexit.o)
                0x80003f5c                atexit
 .text          0x80003f7c        0x0 c:/ti/ccsv5/tools/compiler/gcc-arm-none-eabi-4_7-2012q4/bin/../lib/gcc/arm-none-eabi/4.7.3/../../../../arm-none-eabi/lib\libc.a(lib_a-dtoa.o)
 .text.quorem   0x80003f7c      0x1e0 c:/ti/ccsv5/tools/compiler/gcc-arm-none-eabi-4_7-2012q4/bin/../lib/gcc/arm-none-eabi/4.7.3/../../../../arm-none-eabi/lib\libc.a(lib_a-dtoa.o)
 *fill*         0x8000415c        0x4 00
 .text._dtoa_r  0x80004160     0x1698 c:/ti/ccsv5/tools/compiler/gcc-arm-none-eabi-4_7-2012q4/bin/../lib/gcc/arm-none-eabi/4.7.3/../../../../arm-none-eabi/lib\libc.a(lib_a-dtoa.o)
                0x80004160                _dtoa_r
 .text          0x800057f8        0x0 c:/ti/ccsv5/tools/compiler/gcc-arm-none-eabi-4_7-2012q4/bin/../lib/gcc/arm-none-eabi/4.7.3/../../../../arm-none-eabi/lib\libc.a(lib_a-fflush.o)
 .text._fflush_r
                0x800057f8      0x250 c:/ti/ccsv5/tools/compiler/gcc-arm-none-eabi-4_7-2012q4/bin/../lib/gcc/arm-none-eabi/4.7.3/../../../../arm-none-eabi/lib\libc.a(lib_a-fflush.o)
                0x800057f8                _fflush_r
 .text.fflush   0x80005a48       0x40 c:/ti/ccsv5/tools/compiler/gcc-arm-none-eabi-4_7-2012q4/bin/../lib/gcc/arm-none-eabi/4.7.3/../../../../arm-none-eabi/lib\libc.a(lib_a-fflush.o)
                0x80005a48                fflush
 .text          0x80005a88        0x0 c:/ti/ccsv5/tools/compiler/gcc-arm-none-eabi-4_7-2012q4/bin/../lib/gcc/arm-none-eabi/4.7.3/../../../../arm-none-eabi/lib\libc.a(lib_a-findfp.o)
 .text.__fp_lock
                0x80005a88        0x8 c:/ti/ccsv5/tools/compiler/gcc-arm-none-eabi-4_7-2012q4/bin/../lib/gcc/arm-none-eabi/4.7.3/../../../../arm-none-eabi/lib\libc.a(lib_a-findfp.o)
 .text.__fp_unlock
                0x80005a90        0x8 c:/ti/ccsv5/tools/compiler/gcc-arm-none-eabi-4_7-2012q4/bin/../lib/gcc/arm-none-eabi/4.7.3/../../../../arm-none-eabi/lib\libc.a(lib_a-findfp.o)
 .text._cleanup_r
                0x80005a98       0x18 c:/ti/ccsv5/tools/compiler/gcc-arm-none-eabi-4_7-2012q4/bin/../lib/gcc/arm-none-eabi/4.7.3/../../../../arm-none-eabi/lib\libc.a(lib_a-findfp.o)
                0x80005a98                _cleanup_r
 .text.std.isra.0
                0x80005ab0       0x7c c:/ti/ccsv5/tools/compiler/gcc-arm-none-eabi-4_7-2012q4/bin/../lib/gcc/arm-none-eabi/4.7.3/../../../../arm-none-eabi/lib\libc.a(lib_a-findfp.o)
 .text.__sfmoreglue
                0x80005b2c       0x48 c:/ti/ccsv5/tools/compiler/gcc-arm-none-eabi-4_7-2012q4/bin/../lib/gcc/arm-none-eabi/4.7.3/../../../../arm-none-eabi/lib\libc.a(lib_a-findfp.o)
                0x80005b2c                __sfmoreglue
 .text._cleanup
                0x80005b74       0x10 c:/ti/ccsv5/tools/compiler/gcc-arm-none-eabi-4_7-2012q4/bin/../lib/gcc/arm-none-eabi/4.7.3/../../../../arm-none-eabi/lib\libc.a(lib_a-findfp.o)
                0x80005b74                _cleanup
 .text.__sinit  0x80005b84       0x78 c:/ti/ccsv5/tools/compiler/gcc-arm-none-eabi-4_7-2012q4/bin/../lib/gcc/arm-none-eabi/4.7.3/../../../../arm-none-eabi/lib\libc.a(lib_a-findfp.o)
                0x80005b84                __sinit
 .text.__sfp    0x80005bfc       0xf8 c:/ti/ccsv5/tools/compiler/gcc-arm-none-eabi-4_7-2012q4/bin/../lib/gcc/arm-none-eabi/4.7.3/../../../../arm-none-eabi/lib\libc.a(lib_a-findfp.o)
                0x80005bfc                __sfp
 .text.__sfp_lock_acquire
                0x80005cf4        0x4 c:/ti/ccsv5/tools/compiler/gcc-arm-none-eabi-4_7-2012q4/bin/../lib/gcc/arm-none-eabi/4.7.3/../../../../arm-none-eabi/lib\libc.a(lib_a-findfp.o)
                0x80005cf4                __sfp_lock_acquire
 .text.__sfp_lock_release
                0x80005cf8        0x4 c:/ti/ccsv5/tools/compiler/gcc-arm-none-eabi-4_7-2012q4/bin/../lib/gcc/arm-none-eabi/4.7.3/../../../../arm-none-eabi/lib\libc.a(lib_a-findfp.o)
                0x80005cf8                __sfp_lock_release
 .text.__sinit_lock_acquire
                0x80005cfc        0x4 c:/ti/ccsv5/tools/compiler/gcc-arm-none-eabi-4_7-2012q4/bin/../lib/gcc/arm-none-eabi/4.7.3/../../../../arm-none-eabi/lib\libc.a(lib_a-findfp.o)
                0x80005cfc                __sinit_lock_acquire
 .text.__sinit_lock_release
                0x80005d00        0x4 c:/ti/ccsv5/tools/compiler/gcc-arm-none-eabi-4_7-2012q4/bin/../lib/gcc/arm-none-eabi/4.7.3/../../../../arm-none-eabi/lib\libc.a(lib_a-findfp.o)
                0x80005d00                __sinit_lock_release
 .text.__fp_lock_all
                0x80005d04       0x24 c:/ti/ccsv5/tools/compiler/gcc-arm-none-eabi-4_7-2012q4/bin/../lib/gcc/arm-none-eabi/4.7.3/../../../../arm-none-eabi/lib\libc.a(lib_a-findfp.o)
                0x80005d04                __fp_lock_all
 .text.__fp_unlock_all
                0x80005d28       0x24 c:/ti/ccsv5/tools/compiler/gcc-arm-none-eabi-4_7-2012q4/bin/../lib/gcc/arm-none-eabi/4.7.3/../../../../arm-none-eabi/lib\libc.a(lib_a-findfp.o)
                0x80005d28                __fp_unlock_all
 .text          0x80005d4c        0x0 c:/ti/ccsv5/tools/compiler/gcc-arm-none-eabi-4_7-2012q4/bin/../lib/gcc/arm-none-eabi/4.7.3/../../../../arm-none-eabi/lib\libc.a(lib_a-freer.o)
 .text._malloc_trim_r
                0x80005d4c       0xfc c:/ti/ccsv5/tools/compiler/gcc-arm-none-eabi-4_7-2012q4/bin/../lib/gcc/arm-none-eabi/4.7.3/../../../../arm-none-eabi/lib\libc.a(lib_a-freer.o)
                0x80005d4c                _malloc_trim_r
 .text._free_r  0x80005e48      0x26c c:/ti/ccsv5/tools/compiler/gcc-arm-none-eabi-4_7-2012q4/bin/../lib/gcc/arm-none-eabi/4.7.3/../../../../arm-none-eabi/lib\libc.a(lib_a-freer.o)
                0x80005e48                _free_r
 .text          0x800060b4        0x0 c:/ti/ccsv5/tools/compiler/gcc-arm-none-eabi-4_7-2012q4/bin/../lib/gcc/arm-none-eabi/4.7.3/../../../../arm-none-eabi/lib\libc.a(lib_a-fvwrite.o)
 .text.__sfvwrite_r
                0x800060b4      0x4c4 c:/ti/ccsv5/tools/compiler/gcc-arm-none-eabi-4_7-2012q4/bin/../lib/gcc/arm-none-eabi/4.7.3/../../../../arm-none-eabi/lib\libc.a(lib_a-fvwrite.o)
                0x800060b4                __sfvwrite_r
 .text          0x80006578        0x0 c:/ti/ccsv5/tools/compiler/gcc-arm-none-eabi-4_7-2012q4/bin/../lib/gcc/arm-none-eabi/4.7.3/../../../../arm-none-eabi/lib\libc.a(lib_a-fwalk.o)
 .text._fwalk   0x80006578       0x88 c:/ti/ccsv5/tools/compiler/gcc-arm-none-eabi-4_7-2012q4/bin/../lib/gcc/arm-none-eabi/4.7.3/../../../../arm-none-eabi/lib\libc.a(lib_a-fwalk.o)
                0x80006578                _fwalk
 .text._fwalk_reent
                0x80006600       0x8c c:/ti/ccsv5/tools/compiler/gcc-arm-none-eabi-4_7-2012q4/bin/../lib/gcc/arm-none-eabi/4.7.3/../../../../arm-none-eabi/lib\libc.a(lib_a-fwalk.o)
                0x80006600                _fwalk_reent
 .text          0x8000668c        0x0 c:/ti/ccsv5/tools/compiler/gcc-arm-none-eabi-4_7-2012q4/bin/../lib/gcc/arm-none-eabi/4.7.3/../../../../arm-none-eabi/lib\libc.a(lib_a-locale.o)
 .text._setlocale_r
                0x8000668c       0x6c c:/ti/ccsv5/tools/compiler/gcc-arm-none-eabi-4_7-2012q4/bin/../lib/gcc/arm-none-eabi/4.7.3/../../../../arm-none-eabi/lib\libc.a(lib_a-locale.o)
                0x8000668c                _setlocale_r
 .text.__locale_charset
                0x800066f8        0xc c:/ti/ccsv5/tools/compiler/gcc-arm-none-eabi-4_7-2012q4/bin/../lib/gcc/arm-none-eabi/4.7.3/../../../../arm-none-eabi/lib\libc.a(lib_a-locale.o)
                0x800066f8                __locale_charset
 .text.__locale_mb_cur_max
                0x80006704       0x10 c:/ti/ccsv5/tools/compiler/gcc-arm-none-eabi-4_7-2012q4/bin/../lib/gcc/arm-none-eabi/4.7.3/../../../../arm-none-eabi/lib\libc.a(lib_a-locale.o)
                0x80006704                __locale_mb_cur_max
 .text.__locale_msgcharset
                0x80006714        0xc c:/ti/ccsv5/tools/compiler/gcc-arm-none-eabi-4_7-2012q4/bin/../lib/gcc/arm-none-eabi/4.7.3/../../../../arm-none-eabi/lib\libc.a(lib_a-locale.o)
                0x80006714                __locale_msgcharset
 .text.__locale_cjk_lang
                0x80006720        0x8 c:/ti/ccsv5/tools/compiler/gcc-arm-none-eabi-4_7-2012q4/bin/../lib/gcc/arm-none-eabi/4.7.3/../../../../arm-none-eabi/lib\libc.a(lib_a-locale.o)
                0x80006720                __locale_cjk_lang
 .text._localeconv_r
                0x80006728        0xc c:/ti/ccsv5/tools/compiler/gcc-arm-none-eabi-4_7-2012q4/bin/../lib/gcc/arm-none-eabi/4.7.3/../../../../arm-none-eabi/lib\libc.a(lib_a-locale.o)
                0x80006728                _localeconv_r
 .text.setlocale
                0x80006734       0x1c c:/ti/ccsv5/tools/compiler/gcc-arm-none-eabi-4_7-2012q4/bin/../lib/gcc/arm-none-eabi/4.7.3/../../../../arm-none-eabi/lib\libc.a(lib_a-locale.o)
                0x80006734                setlocale
 .text.localeconv
                0x80006750        0xc c:/ti/ccsv5/tools/compiler/gcc-arm-none-eabi-4_7-2012q4/bin/../lib/gcc/arm-none-eabi/4.7.3/../../../../arm-none-eabi/lib\libc.a(lib_a-locale.o)
                0x80006750                localeconv
 .text          0x8000675c        0x0 c:/ti/ccsv5/tools/compiler/gcc-arm-none-eabi-4_7-2012q4/bin/../lib/gcc/arm-none-eabi/4.7.3/../../../../arm-none-eabi/lib\libc.a(lib_a-makebuf.o)
 .text.__smakebuf_r
                0x8000675c      0x15c c:/ti/ccsv5/tools/compiler/gcc-arm-none-eabi-4_7-2012q4/bin/../lib/gcc/arm-none-eabi/4.7.3/../../../../arm-none-eabi/lib\libc.a(lib_a-makebuf.o)
                0x8000675c                __smakebuf_r
 .text          0x800068b8        0x0 c:/ti/ccsv5/tools/compiler/gcc-arm-none-eabi-4_7-2012q4/bin/../lib/gcc/arm-none-eabi/4.7.3/../../../../arm-none-eabi/lib\libc.a(lib_a-mallocr.o)
 .text._malloc_r
                0x800068b8      0x73c c:/ti/ccsv5/tools/compiler/gcc-arm-none-eabi-4_7-2012q4/bin/../lib/gcc/arm-none-eabi/4.7.3/../../../../arm-none-eabi/lib\libc.a(lib_a-mallocr.o)
                0x800068b8                _malloc_r
 .text          0x80006ff4        0x0 c:/ti/ccsv5/tools/compiler/gcc-arm-none-eabi-4_7-2012q4/bin/../lib/gcc/arm-none-eabi/4.7.3/../../../../arm-none-eabi/lib\libc.a(lib_a-memchr.o)
 .text.memchr   0x80006ff4      0x11c c:/ti/ccsv5/tools/compiler/gcc-arm-none-eabi-4_7-2012q4/bin/../lib/gcc/arm-none-eabi/4.7.3/../../../../arm-none-eabi/lib\libc.a(lib_a-memchr.o)
                0x80006ff4                memchr
 .text          0x80007110        0x0 c:/ti/ccsv5/tools/compiler/gcc-arm-none-eabi-4_7-2012q4/bin/../lib/gcc/arm-none-eabi/4.7.3/../../../../arm-none-eabi/lib\libc.a(lib_a-memcpy.o)
 .text.memcpy   0x80007110       0xf4 c:/ti/ccsv5/tools/compiler/gcc-arm-none-eabi-4_7-2012q4/bin/../lib/gcc/arm-none-eabi/4.7.3/../../../../arm-none-eabi/lib\libc.a(lib_a-memcpy.o)
                0x80007110                memcpy
 .text          0x80007204        0x0 c:/ti/ccsv5/tools/compiler/gcc-arm-none-eabi-4_7-2012q4/bin/../lib/gcc/arm-none-eabi/4.7.3/../../../../arm-none-eabi/lib\libc.a(lib_a-memmove.o)
 .text.memmove  0x80007204      0x134 c:/ti/ccsv5/tools/compiler/gcc-arm-none-eabi-4_7-2012q4/bin/../lib/gcc/arm-none-eabi/4.7.3/../../../../arm-none-eabi/lib\libc.a(lib_a-memmove.o)
                0x80007204                memmove
 .text          0x80007338        0x0 c:/ti/ccsv5/tools/compiler/gcc-arm-none-eabi-4_7-2012q4/bin/../lib/gcc/arm-none-eabi/4.7.3/../../../../arm-none-eabi/lib\libc.a(lib_a-mlock.o)
 .text.__malloc_lock
                0x80007338        0x4 c:/ti/ccsv5/tools/compiler/gcc-arm-none-eabi-4_7-2012q4/bin/../lib/gcc/arm-none-eabi/4.7.3/../../../../arm-none-eabi/lib\libc.a(lib_a-mlock.o)
                0x80007338                __malloc_lock
 .text.__malloc_unlock
                0x8000733c        0x4 c:/ti/ccsv5/tools/compiler/gcc-arm-none-eabi-4_7-2012q4/bin/../lib/gcc/arm-none-eabi/4.7.3/../../../../arm-none-eabi/lib\libc.a(lib_a-mlock.o)
                0x8000733c                __malloc_unlock
 .text          0x80007340        0x0 c:/ti/ccsv5/tools/compiler/gcc-arm-none-eabi-4_7-2012q4/bin/../lib/gcc/arm-none-eabi/4.7.3/../../../../arm-none-eabi/lib\libc.a(lib_a-mprec.o)
 .text._Balloc  0x80007340       0x8c c:/ti/ccsv5/tools/compiler/gcc-arm-none-eabi-4_7-2012q4/bin/../lib/gcc/arm-none-eabi/4.7.3/../../../../arm-none-eabi/lib\libc.a(lib_a-mprec.o)
                0x80007340                _Balloc
 .text._Bfree   0x800073cc       0x1c c:/ti/ccsv5/tools/compiler/gcc-arm-none-eabi-4_7-2012q4/bin/../lib/gcc/arm-none-eabi/4.7.3/../../../../arm-none-eabi/lib\libc.a(lib_a-mprec.o)
                0x800073cc                _Bfree
 .text.__multadd
                0x800073e8       0xdc c:/ti/ccsv5/tools/compiler/gcc-arm-none-eabi-4_7-2012q4/bin/../lib/gcc/arm-none-eabi/4.7.3/../../../../arm-none-eabi/lib\libc.a(lib_a-mprec.o)
                0x800073e8                __multadd
 .text.__s2b    0x800074c4       0xf0 c:/ti/ccsv5/tools/compiler/gcc-arm-none-eabi-4_7-2012q4/bin/../lib/gcc/arm-none-eabi/4.7.3/../../../../arm-none-eabi/lib\libc.a(lib_a-mprec.o)
                0x800074c4                __s2b
 .text.__hi0bits
                0x800075b4       0x50 c:/ti/ccsv5/tools/compiler/gcc-arm-none-eabi-4_7-2012q4/bin/../lib/gcc/arm-none-eabi/4.7.3/../../../../arm-none-eabi/lib\libc.a(lib_a-mprec.o)
                0x800075b4                __hi0bits
 .text.__lo0bits
                0x80007604       0x94 c:/ti/ccsv5/tools/compiler/gcc-arm-none-eabi-4_7-2012q4/bin/../lib/gcc/arm-none-eabi/4.7.3/../../../../arm-none-eabi/lib\libc.a(lib_a-mprec.o)
                0x80007604                __lo0bits
 .text.__i2b    0x80007698       0x24 c:/ti/ccsv5/tools/compiler/gcc-arm-none-eabi-4_7-2012q4/bin/../lib/gcc/arm-none-eabi/4.7.3/../../../../arm-none-eabi/lib\libc.a(lib_a-mprec.o)
                0x80007698                __i2b
 .text.__multiply
                0x800076bc      0x1e4 c:/ti/ccsv5/tools/compiler/gcc-arm-none-eabi-4_7-2012q4/bin/../lib/gcc/arm-none-eabi/4.7.3/../../../../arm-none-eabi/lib\libc.a(lib_a-mprec.o)
                0x800076bc                __multiply
 .text.__pow5mult
                0x800078a0       0xf4 c:/ti/ccsv5/tools/compiler/gcc-arm-none-eabi-4_7-2012q4/bin/../lib/gcc/arm-none-eabi/4.7.3/../../../../arm-none-eabi/lib\libc.a(lib_a-mprec.o)
                0x800078a0                __pow5mult
 .text.__lshift
                0x80007994      0x104 c:/ti/ccsv5/tools/compiler/gcc-arm-none-eabi-4_7-2012q4/bin/../lib/gcc/arm-none-eabi/4.7.3/../../../../arm-none-eabi/lib\libc.a(lib_a-mprec.o)
                0x80007994                __lshift
 .text.__mcmp   0x80007a98       0x64 c:/ti/ccsv5/tools/compiler/gcc-arm-none-eabi-4_7-2012q4/bin/../lib/gcc/arm-none-eabi/4.7.3/../../../../arm-none-eabi/lib\libc.a(lib_a-mprec.o)
                0x80007a98                __mcmp
 .text.__mdiff  0x80007afc      0x14c c:/ti/ccsv5/tools/compiler/gcc-arm-none-eabi-4_7-2012q4/bin/../lib/gcc/arm-none-eabi/4.7.3/../../../../arm-none-eabi/lib\libc.a(lib_a-mprec.o)
                0x80007afc                __mdiff
 .text.__ulp    0x80007c48       0x64 c:/ti/ccsv5/tools/compiler/gcc-arm-none-eabi-4_7-2012q4/bin/../lib/gcc/arm-none-eabi/4.7.3/../../../../arm-none-eabi/lib\libc.a(lib_a-mprec.o)
                0x80007c48                __ulp
 .text.__b2d    0x80007cac       0xcc c:/ti/ccsv5/tools/compiler/gcc-arm-none-eabi-4_7-2012q4/bin/../lib/gcc/arm-none-eabi/4.7.3/../../../../arm-none-eabi/lib\libc.a(lib_a-mprec.o)
                0x80007cac                __b2d
 .text.__d2b    0x80007d78      0x108 c:/ti/ccsv5/tools/compiler/gcc-arm-none-eabi-4_7-2012q4/bin/../lib/gcc/arm-none-eabi/4.7.3/../../../../arm-none-eabi/lib\libc.a(lib_a-mprec.o)
                0x80007d78                __d2b
 .text.__ratio  0x80007e80       0x90 c:/ti/ccsv5/tools/compiler/gcc-arm-none-eabi-4_7-2012q4/bin/../lib/gcc/arm-none-eabi/4.7.3/../../../../arm-none-eabi/lib\libc.a(lib_a-mprec.o)
                0x80007e80                __ratio
 .text._mprec_log10
                0x80007f10       0x50 c:/ti/ccsv5/tools/compiler/gcc-arm-none-eabi-4_7-2012q4/bin/../lib/gcc/arm-none-eabi/4.7.3/../../../../arm-none-eabi/lib\libc.a(lib_a-mprec.o)
                0x80007f10                _mprec_log10
 .text.__copybits
                0x80007f60       0x74 c:/ti/ccsv5/tools/compiler/gcc-arm-none-eabi-4_7-2012q4/bin/../lib/gcc/arm-none-eabi/4.7.3/../../../../arm-none-eabi/lib\libc.a(lib_a-mprec.o)
                0x80007f60                __copybits
 .text.__any_on
                0x80007fd4       0x88 c:/ti/ccsv5/tools/compiler/gcc-arm-none-eabi-4_7-2012q4/bin/../lib/gcc/arm-none-eabi/4.7.3/../../../../arm-none-eabi/lib\libc.a(lib_a-mprec.o)
                0x80007fd4                __any_on
 .text          0x8000805c        0x0 c:/ti/ccsv5/tools/compiler/gcc-arm-none-eabi-4_7-2012q4/bin/../lib/gcc/arm-none-eabi/4.7.3/../../../../arm-none-eabi/lib\libc.a(lib_a-reallocr.o)
 .text._realloc_r
                0x8000805c      0x574 c:/ti/ccsv5/tools/compiler/gcc-arm-none-eabi-4_7-2012q4/bin/../lib/gcc/arm-none-eabi/4.7.3/../../../../arm-none-eabi/lib\libc.a(lib_a-reallocr.o)
                0x8000805c                _realloc_r
 .text          0x800085d0        0x0 c:/ti/ccsv5/tools/compiler/gcc-arm-none-eabi-4_7-2012q4/bin/../lib/gcc/arm-none-eabi/4.7.3/../../../../arm-none-eabi/lib\libc.a(lib_a-s_fpclassify.o)
 .text.__fpclassifyd
                0x800085d0       0x6c c:/ti/ccsv5/tools/compiler/gcc-arm-none-eabi-4_7-2012q4/bin/../lib/gcc/arm-none-eabi/4.7.3/../../../../arm-none-eabi/lib\libc.a(lib_a-s_fpclassify.o)
                0x800085d0                __fpclassifyd
 .text          0x8000863c        0x0 c:/ti/ccsv5/tools/compiler/gcc-arm-none-eabi-4_7-2012q4/bin/../lib/gcc/arm-none-eabi/4.7.3/../../../../arm-none-eabi/lib\libc.a(lib_a-sbrkr.o)
 .text._sbrk_r  0x8000863c       0x40 c:/ti/ccsv5/tools/compiler/gcc-arm-none-eabi-4_7-2012q4/bin/../lib/gcc/arm-none-eabi/4.7.3/../../../../arm-none-eabi/lib\libc.a(lib_a-sbrkr.o)
                0x8000863c                _sbrk_r
 .text          0x8000867c        0x0 c:/ti/ccsv5/tools/compiler/gcc-arm-none-eabi-4_7-2012q4/bin/../lib/gcc/arm-none-eabi/4.7.3/../../../../arm-none-eabi/lib\libc.a(lib_a-stdio.o)
 .text.__sread  0x8000867c       0x34 c:/ti/ccsv5/tools/compiler/gcc-arm-none-eabi-4_7-2012q4/bin/../lib/gcc/arm-none-eabi/4.7.3/../../../../arm-none-eabi/lib\libc.a(lib_a-stdio.o)
                0x8000867c                __sread
 .text.__seofread
                0x800086b0        0x8 c:/ti/ccsv5/tools/compiler/gcc-arm-none-eabi-4_7-2012q4/bin/../lib/gcc/arm-none-eabi/4.7.3/../../../../arm-none-eabi/lib\libc.a(lib_a-stdio.o)
                0x800086b0                __seofread
 .text.__swrite
                0x800086b8       0x58 c:/ti/ccsv5/tools/compiler/gcc-arm-none-eabi-4_7-2012q4/bin/../lib/gcc/arm-none-eabi/4.7.3/../../../../arm-none-eabi/lib\libc.a(lib_a-stdio.o)
                0x800086b8                __swrite
 .text.__sseek  0x80008710       0x34 c:/ti/ccsv5/tools/compiler/gcc-arm-none-eabi-4_7-2012q4/bin/../lib/gcc/arm-none-eabi/4.7.3/../../../../arm-none-eabi/lib\libc.a(lib_a-stdio.o)
                0x80008710                __sseek
 .text.__sclose
                0x80008744       0x14 c:/ti/ccsv5/tools/compiler/gcc-arm-none-eabi-4_7-2012q4/bin/../lib/gcc/arm-none-eabi/4.7.3/../../../../arm-none-eabi/lib\libc.a(lib_a-stdio.o)
                0x80008744                __sclose
 .text          0x80008758        0x0 c:/ti/ccsv5/tools/compiler/gcc-arm-none-eabi-4_7-2012q4/bin/../lib/gcc/arm-none-eabi/4.7.3/../../../../arm-none-eabi/lib\libc.a(lib_a-strcmp.o)
 .text.strcmp   0x80008758       0x94 c:/ti/ccsv5/tools/compiler/gcc-arm-none-eabi-4_7-2012q4/bin/../lib/gcc/arm-none-eabi/4.7.3/../../../../arm-none-eabi/lib\libc.a(lib_a-strcmp.o)
                0x80008758                strcmp
 .text.strcmp_unaligned
                0x800087ec      0x19c c:/ti/ccsv5/tools/compiler/gcc-arm-none-eabi-4_7-2012q4/bin/../lib/gcc/arm-none-eabi/4.7.3/../../../../arm-none-eabi/lib\libc.a(lib_a-strcmp.o)
 .text          0x80008988        0x0 c:/ti/ccsv5/tools/compiler/gcc-arm-none-eabi-4_7-2012q4/bin/../lib/gcc/arm-none-eabi/4.7.3/../../../../arm-none-eabi/lib\libc.a(lib_a-vfiprintf.o)
 .text.__sprint_r
                0x80008988       0xc0 c:/ti/ccsv5/tools/compiler/gcc-arm-none-eabi-4_7-2012q4/bin/../lib/gcc/arm-none-eabi/4.7.3/../../../../arm-none-eabi/lib\libc.a(lib_a-vfiprintf.o)
                0x80008988                __sprint_r
 .text._vfiprintf_r
                0x80008a48     0x11e0 c:/ti/ccsv5/tools/compiler/gcc-arm-none-eabi-4_7-2012q4/bin/../lib/gcc/arm-none-eabi/4.7.3/../../../../arm-none-eabi/lib\libc.a(lib_a-vfiprintf.o)
                0x80008a48                _vfiprintf_r
 .text.vfiprintf
                0x80009c28       0x2c c:/ti/ccsv5/tools/compiler/gcc-arm-none-eabi-4_7-2012q4/bin/../lib/gcc/arm-none-eabi/4.7.3/../../../../arm-none-eabi/lib\libc.a(lib_a-vfiprintf.o)
                0x80009c28                vfiprintf
 .text          0x80009c54        0x0 c:/ti/ccsv5/tools/compiler/gcc-arm-none-eabi-4_7-2012q4/bin/../lib/gcc/arm-none-eabi/4.7.3/../../../../arm-none-eabi/lib\libc.a(lib_a-writer.o)
 .text._write_r
                0x80009c54       0x44 c:/ti/ccsv5/tools/compiler/gcc-arm-none-eabi-4_7-2012q4/bin/../lib/gcc/arm-none-eabi/4.7.3/../../../../arm-none-eabi/lib\libc.a(lib_a-writer.o)
                0x80009c54                _write_r
 .text          0x80009c98        0x0 c:/ti/ccsv5/tools/compiler/gcc-arm-none-eabi-4_7-2012q4/bin/../lib/gcc/arm-none-eabi/4.7.3/../../../../arm-none-eabi/lib\libc.a(lib_a-callocr.o)
 .text._calloc_r
                0x80009c98       0x94 c:/ti/ccsv5/tools/compiler/gcc-arm-none-eabi-4_7-2012q4/bin/../lib/gcc/arm-none-eabi/4.7.3/../../../../arm-none-eabi/lib\libc.a(lib_a-callocr.o)
                0x80009c98                _calloc_r
 .text          0x80009d2c        0x0 c:/ti/ccsv5/tools/compiler/gcc-arm-none-eabi-4_7-2012q4/bin/../lib/gcc/arm-none-eabi/4.7.3/../../../../arm-none-eabi/lib\libc.a(lib_a-closer.o)
 .text._close_r
                0x80009d2c       0x3c c:/ti/ccsv5/tools/compiler/gcc-arm-none-eabi-4_7-2012q4/bin/../lib/gcc/arm-none-eabi/4.7.3/../../../../arm-none-eabi/lib\libc.a(lib_a-closer.o)
                0x80009d2c                _close_r
 .text          0x80009d68        0x0 c:/ti/ccsv5/tools/compiler/gcc-arm-none-eabi-4_7-2012q4/bin/../lib/gcc/arm-none-eabi/4.7.3/../../../../arm-none-eabi/lib\libc.a(lib_a-fclose.o)
 .text._fclose_r
                0x80009d68       0xf8 c:/ti/ccsv5/tools/compiler/gcc-arm-none-eabi-4_7-2012q4/bin/../lib/gcc/arm-none-eabi/4.7.3/../../../../arm-none-eabi/lib\libc.a(lib_a-fclose.o)
                0x80009d68                _fclose_r
 .text.fclose   0x80009e60       0x14 c:/ti/ccsv5/tools/compiler/gcc-arm-none-eabi-4_7-2012q4/bin/../lib/gcc/arm-none-eabi/4.7.3/../../../../arm-none-eabi/lib\libc.a(lib_a-fclose.o)
                0x80009e60                fclose
 .text          0x80009e74        0x0 c:/ti/ccsv5/tools/compiler/gcc-arm-none-eabi-4_7-2012q4/bin/../lib/gcc/arm-none-eabi/4.7.3/../../../../arm-none-eabi/lib\libc.a(lib_a-fputwc.o)
 .text._fputwc_r
                0x80009e74      0x150 c:/ti/ccsv5/tools/compiler/gcc-arm-none-eabi-4_7-2012q4/bin/../lib/gcc/arm-none-eabi/4.7.3/../../../../arm-none-eabi/lib\libc.a(lib_a-fputwc.o)
                0x80009e74                _fputwc_r
 .text.fputwc   0x80009fc4       0x4c c:/ti/ccsv5/tools/compiler/gcc-arm-none-eabi-4_7-2012q4/bin/../lib/gcc/arm-none-eabi/4.7.3/../../../../arm-none-eabi/lib\libc.a(lib_a-fputwc.o)
                0x80009fc4                fputwc
 .text          0x8000a010        0x0 c:/ti/ccsv5/tools/compiler/gcc-arm-none-eabi-4_7-2012q4/bin/../lib/gcc/arm-none-eabi/4.7.3/../../../../arm-none-eabi/lib\libc.a(lib_a-fstatr.o)
 .text._fstat_r
                0x8000a010       0x40 c:/ti/ccsv5/tools/compiler/gcc-arm-none-eabi-4_7-2012q4/bin/../lib/gcc/arm-none-eabi/4.7.3/../../../../arm-none-eabi/lib\libc.a(lib_a-fstatr.o)
                0x8000a010                _fstat_r
 .text          0x8000a050        0x0 c:/ti/ccsv5/tools/compiler/gcc-arm-none-eabi-4_7-2012q4/bin/../lib/gcc/arm-none-eabi/4.7.3/../../../../arm-none-eabi/lib\libc.a(lib_a-isattyr.o)
 .text._isatty_r
                0x8000a050       0x3c c:/ti/ccsv5/tools/compiler/gcc-arm-none-eabi-4_7-2012q4/bin/../lib/gcc/arm-none-eabi/4.7.3/../../../../arm-none-eabi/lib\libc.a(lib_a-isattyr.o)
                0x8000a050                _isatty_r
 .text          0x8000a08c        0x0 c:/ti/ccsv5/tools/compiler/gcc-arm-none-eabi-4_7-2012q4/bin/../lib/gcc/arm-none-eabi/4.7.3/../../../../arm-none-eabi/lib\libc.a(lib_a-lseekr.o)
 .text._lseek_r
                0x8000a08c       0x44 c:/ti/ccsv5/tools/compiler/gcc-arm-none-eabi-4_7-2012q4/bin/../lib/gcc/arm-none-eabi/4.7.3/../../../../arm-none-eabi/lib\libc.a(lib_a-lseekr.o)
                0x8000a08c                _lseek_r
 .text          0x8000a0d0        0x0 c:/ti/ccsv5/tools/compiler/gcc-arm-none-eabi-4_7-2012q4/bin/../lib/gcc/arm-none-eabi/4.7.3/../../../../arm-none-eabi/lib\libc.a(lib_a-readr.o)
 .text._read_r  0x8000a0d0       0x44 c:/ti/ccsv5/tools/compiler/gcc-arm-none-eabi-4_7-2012q4/bin/../lib/gcc/arm-none-eabi/4.7.3/../../../../arm-none-eabi/lib\libc.a(lib_a-readr.o)
                0x8000a0d0                _read_r
 .text          0x8000a114        0x0 c:/ti/ccsv5/tools/compiler/gcc-arm-none-eabi-4_7-2012q4/bin/../lib/gcc/arm-none-eabi/4.7.3/../../../../arm-none-eabi/lib\libc.a(lib_a-reent.o)
 .text.cleanup_glue
                0x8000a114       0x2c c:/ti/ccsv5/tools/compiler/gcc-arm-none-eabi-4_7-2012q4/bin/../lib/gcc/arm-none-eabi/4.7.3/../../../../arm-none-eabi/lib\libc.a(lib_a-reent.o)
                0x8000a114                cleanup_glue
 .text._reclaim_reent
                0x8000a140       0xfc c:/ti/ccsv5/tools/compiler/gcc-arm-none-eabi-4_7-2012q4/bin/../lib/gcc/arm-none-eabi/4.7.3/../../../../arm-none-eabi/lib\libc.a(lib_a-reent.o)
                0x8000a140                _reclaim_reent
 .text._wrapup_reent
                0x8000a23c       0x74 c:/ti/ccsv5/tools/compiler/gcc-arm-none-eabi-4_7-2012q4/bin/../lib/gcc/arm-none-eabi/4.7.3/../../../../arm-none-eabi/lib\libc.a(lib_a-reent.o)
                0x8000a23c                _wrapup_reent
 .text          0x8000a2b0        0x0 c:/ti/ccsv5/tools/compiler/gcc-arm-none-eabi-4_7-2012q4/bin/../lib/gcc/arm-none-eabi/4.7.3/../../../../arm-none-eabi/lib\libc.a(lib_a-wbuf.o)
 .text.__swbuf_r
                0x8000a2b0      0x130 c:/ti/ccsv5/tools/compiler/gcc-arm-none-eabi-4_7-2012q4/bin/../lib/gcc/arm-none-eabi/4.7.3/../../../../arm-none-eabi/lib\libc.a(lib_a-wbuf.o)
                0x8000a2b0                __swbuf_r
 .text.__swbuf  0x8000a3e0       0x1c c:/ti/ccsv5/tools/compiler/gcc-arm-none-eabi-4_7-2012q4/bin/../lib/gcc/arm-none-eabi/4.7.3/../../../../arm-none-eabi/lib\libc.a(lib_a-wbuf.o)
                0x8000a3e0                __swbuf
 .text          0x8000a3fc        0x0 c:/ti/ccsv5/tools/compiler/gcc-arm-none-eabi-4_7-2012q4/bin/../lib/gcc/arm-none-eabi/4.7.3/../../../../arm-none-eabi/lib\libc.a(lib_a-wcrtomb.o)
 .text._wcrtomb_r
                0x8000a3fc       0x90 c:/ti/ccsv5/tools/compiler/gcc-arm-none-eabi-4_7-2012q4/bin/../lib/gcc/arm-none-eabi/4.7.3/../../../../arm-none-eabi/lib\libc.a(lib_a-wcrtomb.o)
                0x8000a3fc                _wcrtomb_r
 .text.wcrtomb  0x8000a48c       0xa4 c:/ti/ccsv5/tools/compiler/gcc-arm-none-eabi-4_7-2012q4/bin/../lib/gcc/arm-none-eabi/4.7.3/../../../../arm-none-eabi/lib\libc.a(lib_a-wcrtomb.o)
                0x8000a48c                wcrtomb
 .text          0x8000a530        0x0 c:/ti/ccsv5/tools/compiler/gcc-arm-none-eabi-4_7-2012q4/bin/../lib/gcc/arm-none-eabi/4.7.3/../../../../arm-none-eabi/lib\libc.a(lib_a-wctomb_r.o)
 .text.__ascii_wctomb
                0x8000a530       0x2c c:/ti/ccsv5/tools/compiler/gcc-arm-none-eabi-4_7-2012q4/bin/../lib/gcc/arm-none-eabi/4.7.3/../../../../arm-none-eabi/lib\libc.a(lib_a-wctomb_r.o)
                0x8000a530                __ascii_wctomb
 .text._wctomb_r
                0x8000a55c       0x50 c:/ti/ccsv5/tools/compiler/gcc-arm-none-eabi-4_7-2012q4/bin/../lib/gcc/arm-none-eabi/4.7.3/../../../../arm-none-eabi/lib\libc.a(lib_a-wctomb_r.o)
                0x8000a55c                _wctomb_r
 .text          0x8000a5ac      0x114 c:/ti/ccsv5/tools/compiler/gcc-arm-none-eabi-4_7-2012q4/bin/../lib/gcc/arm-none-eabi/4.7.3\libgcc.a(_udivsi3.o)
                0x8000a5ac                __aeabi_uidiv
                0x8000a5ac                __udivsi3
                0x8000a6a0                __aeabi_uidivmod
 .text          0x8000a6c0        0x4 c:/ti/ccsv5/tools/compiler/gcc-arm-none-eabi-4_7-2012q4/bin/../lib/gcc/arm-none-eabi/4.7.3\libgcc.a(_dvmd_tls.o)
                0x8000a6c0                __aeabi_idiv0
                0x8000a6c0                __aeabi_ldiv0
 .text          0x8000a6c4      0x41c c:/ti/ccsv5/tools/compiler/gcc-arm-none-eabi-4_7-2012q4/bin/../lib/gcc/arm-none-eabi/4.7.3\libgcc.a(_arm_addsubdf3.o)
                0x8000a6c4                __aeabi_drsub
                0x8000a6cc                __aeabi_dsub
                0x8000a6cc                __subdf3
                0x8000a6d0                __aeabi_dadd
                0x8000a6d0                __adddf3
                0x8000a9e0                __floatunsidf
                0x8000a9e0                __aeabi_ui2d
                0x8000aa04                __floatsidf
                0x8000aa04                __aeabi_i2d
                0x8000aa2c                __aeabi_f2d
                0x8000aa2c                __extendsfdf2
                0x8000aa6c                __floatundidf
                0x8000aa6c                __aeabi_ul2d
                0x8000aa80                __floatdidf
                0x8000aa80                __aeabi_l2d
 .text          0x8000aae0      0x49c c:/ti/ccsv5/tools/compiler/gcc-arm-none-eabi-4_7-2012q4/bin/../lib/gcc/arm-none-eabi/4.7.3\libgcc.a(_arm_muldivdf3.o)
                0x8000aae0                __aeabi_dmul
                0x8000aae0                __muldf3
                0x8000ad70                __divdf3
                0x8000ad70                __aeabi_ddiv
 .text          0x8000af7c      0x144 c:/ti/ccsv5/tools/compiler/gcc-arm-none-eabi-4_7-2012q4/bin/../lib/gcc/arm-none-eabi/4.7.3\libgcc.a(_arm_cmpdf2.o)
                0x8000af7c                __gtdf2
                0x8000af7c                __gedf2
                0x8000af84                __ltdf2
                0x8000af84                __ledf2
                0x8000af8c                __nedf2
                0x8000af8c                __eqdf2
                0x8000af8c                __cmpdf2
                0x8000b014                __aeabi_cdrcmple
                0x8000b030                __aeabi_cdcmpeq
                0x8000b030                __aeabi_cdcmple
                0x8000b048                __aeabi_dcmpeq
                0x8000b060                __aeabi_dcmplt
                0x8000b078                __aeabi_dcmple
                0x8000b090                __aeabi_dcmpge
                0x8000b0a8                __aeabi_dcmpgt
 .text          0x8000b0c0       0x5c c:/ti/ccsv5/tools/compiler/gcc-arm-none-eabi-4_7-2012q4/bin/../lib/gcc/arm-none-eabi/4.7.3\libgcc.a(_arm_fixdfsi.o)
                0x8000b0c0                __aeabi_d2iz
                0x8000b0c0                __fixdfsi
 .text          0x8000b11c       0x3c c:/ti/ccsv5/tools/compiler/gcc-arm-none-eabi-4_7-2012q4/bin/../lib/gcc/arm-none-eabi/4.7.3\libgcc.a(_aeabi_uldivmod.o)
                0x8000b11c                __aeabi_uldivmod
 .text          0x8000b158       0x84 c:/ti/ccsv5/tools/compiler/gcc-arm-none-eabi-4_7-2012q4/bin/../lib/gcc/arm-none-eabi/4.7.3\libgcc.a(bpabi.o)
                0x8000b158                __gnu_ldivmod_helper
                0x8000b19c                __gnu_uldivmod_helper
 .text          0x8000b1dc      0x4f0 c:/ti/ccsv5/tools/compiler/gcc-arm-none-eabi-4_7-2012q4/bin/../lib/gcc/arm-none-eabi/4.7.3\libgcc.a(_divdi3.o)
                0x8000b1dc                __divdi3
 .text          0x8000b6cc      0x488 c:/ti/ccsv5/tools/compiler/gcc-arm-none-eabi-4_7-2012q4/bin/../lib/gcc/arm-none-eabi/4.7.3\libgcc.a(_udivdi3.o)
                0x8000b6cc                __udivdi3
 .text          0x8000bb54       0x48 c:/ti/ccsv5/tools/compiler/gcc-arm-none-eabi-4_7-2012q4/bin/../lib/gcc/arm-none-eabi/4.7.3\libgcc.a(_clzsi2.o)
                0x8000bb54                __clzsi2
 .text          0x8000bb9c        0x0 c:/ti/ccsv5/tools/compiler/gcc-arm-none-eabi-4_7-2012q4/bin/../lib/gcc/arm-none-eabi/4.7.3/../../../../arm-none-eabi/lib\librdimon.a(rdimon-syscalls.o)
 .text.error    0x8000bb9c       0x38 c:/ti/ccsv5/tools/compiler/gcc-arm-none-eabi-4_7-2012q4/bin/../lib/gcc/arm-none-eabi/4.7.3/../../../../arm-none-eabi/lib\librdimon.a(rdimon-syscalls.o)
 .text.findslot
                0x8000bbd4       0x68 c:/ti/ccsv5/tools/compiler/gcc-arm-none-eabi-4_7-2012q4/bin/../lib/gcc/arm-none-eabi/4.7.3/../../../../arm-none-eabi/lib\librdimon.a(rdimon-syscalls.o)
 .text.checkerror
                0x8000bc3c        0xc c:/ti/ccsv5/tools/compiler/gcc-arm-none-eabi-4_7-2012q4/bin/../lib/gcc/arm-none-eabi/4.7.3/../../../../arm-none-eabi/lib\librdimon.a(rdimon-syscalls.o)
 .text.initialise_monitor_handles
                0x8000bc48       0xf8 c:/ti/ccsv5/tools/compiler/gcc-arm-none-eabi-4_7-2012q4/bin/../lib/gcc/arm-none-eabi/4.7.3/../../../../arm-none-eabi/lib\librdimon.a(rdimon-syscalls.o)
                0x8000bc48                initialise_monitor_handles
 .text._swiread
                0x8000bd40       0x38 c:/ti/ccsv5/tools/compiler/gcc-arm-none-eabi-4_7-2012q4/bin/../lib/gcc/arm-none-eabi/4.7.3/../../../../arm-none-eabi/lib\librdimon.a(rdimon-syscalls.o)
                0x8000bd40                _swiread
 .text._read    0x8000bd78       0x58 c:/ti/ccsv5/tools/compiler/gcc-arm-none-eabi-4_7-2012q4/bin/../lib/gcc/arm-none-eabi/4.7.3/../../../../arm-none-eabi/lib\librdimon.a(rdimon-syscalls.o)
                0x8000bd78                _read
 .text._swilseek
                0x8000bdd0       0xe8 c:/ti/ccsv5/tools/compiler/gcc-arm-none-eabi-4_7-2012q4/bin/../lib/gcc/arm-none-eabi/4.7.3/../../../../arm-none-eabi/lib\librdimon.a(rdimon-syscalls.o)
                0x8000bdd0                _swilseek
 .text._lseek   0x8000beb8        0x4 c:/ti/ccsv5/tools/compiler/gcc-arm-none-eabi-4_7-2012q4/bin/../lib/gcc/arm-none-eabi/4.7.3/../../../../arm-none-eabi/lib\librdimon.a(rdimon-syscalls.o)
                0x8000beb8                _lseek
 .text._swiwrite
                0x8000bebc       0x38 c:/ti/ccsv5/tools/compiler/gcc-arm-none-eabi-4_7-2012q4/bin/../lib/gcc/arm-none-eabi/4.7.3/../../../../arm-none-eabi/lib\librdimon.a(rdimon-syscalls.o)
                0x8000bebc                _swiwrite
 .text._write   0x8000bef4       0x78 c:/ti/ccsv5/tools/compiler/gcc-arm-none-eabi-4_7-2012q4/bin/../lib/gcc/arm-none-eabi/4.7.3/../../../../arm-none-eabi/lib\librdimon.a(rdimon-syscalls.o)
                0x8000bef4                _write
 .text._swiclose
                0x8000bf6c       0x38 c:/ti/ccsv5/tools/compiler/gcc-arm-none-eabi-4_7-2012q4/bin/../lib/gcc/arm-none-eabi/4.7.3/../../../../arm-none-eabi/lib\librdimon.a(rdimon-syscalls.o)
                0x8000bf6c                _swiclose
 .text._close   0x8000bfa4       0x78 c:/ti/ccsv5/tools/compiler/gcc-arm-none-eabi-4_7-2012q4/bin/../lib/gcc/arm-none-eabi/4.7.3/../../../../arm-none-eabi/lib\librdimon.a(rdimon-syscalls.o)
                0x8000bfa4                _close
 .text._getpid  0x8000c01c        0x8 c:/ti/ccsv5/tools/compiler/gcc-arm-none-eabi-4_7-2012q4/bin/../lib/gcc/arm-none-eabi/4.7.3/../../../../arm-none-eabi/lib\librdimon.a(rdimon-syscalls.o)
                0x8000c01c                _getpid
 .text._sbrk    0x8000c024       0x54 c:/ti/ccsv5/tools/compiler/gcc-arm-none-eabi-4_7-2012q4/bin/../lib/gcc/arm-none-eabi/4.7.3/../../../../arm-none-eabi/lib\librdimon.a(rdimon-syscalls.o)
                0x8000c024                _sbrk
 .text._swistat
                0x8000c078       0x6c c:/ti/ccsv5/tools/compiler/gcc-arm-none-eabi-4_7-2012q4/bin/../lib/gcc/arm-none-eabi/4.7.3/../../../../arm-none-eabi/lib\librdimon.a(rdimon-syscalls.o)
                0x8000c078                _swistat
 .text._fstat   0x8000c0e4       0x2c c:/ti/ccsv5/tools/compiler/gcc-arm-none-eabi-4_7-2012q4/bin/../lib/gcc/arm-none-eabi/4.7.3/../../../../arm-none-eabi/lib\librdimon.a(rdimon-syscalls.o)
                0x8000c0e4                _fstat
 .text._stat    0x8000c110       0x68 c:/ti/ccsv5/tools/compiler/gcc-arm-none-eabi-4_7-2012q4/bin/../lib/gcc/arm-none-eabi/4.7.3/../../../../arm-none-eabi/lib\librdimon.a(rdimon-syscalls.o)
                0x8000c110                _stat
 .text._swiopen
                0x8000c178      0x114 c:/ti/ccsv5/tools/compiler/gcc-arm-none-eabi-4_7-2012q4/bin/../lib/gcc/arm-none-eabi/4.7.3/../../../../arm-none-eabi/lib\librdimon.a(rdimon-syscalls.o)
                0x8000c178                _swiopen
 .text._open    0x8000c28c       0x1c c:/ti/ccsv5/tools/compiler/gcc-arm-none-eabi-4_7-2012q4/bin/../lib/gcc/arm-none-eabi/4.7.3/../../../../arm-none-eabi/lib\librdimon.a(rdimon-syscalls.o)
                0x8000c28c                _open
 .text._link    0x8000c2a8       0x1c c:/ti/ccsv5/tools/compiler/gcc-arm-none-eabi-4_7-2012q4/bin/../lib/gcc/arm-none-eabi/4.7.3/../../../../arm-none-eabi/lib\librdimon.a(rdimon-syscalls.o)
                0x8000c2a8                _link
 .text._unlink  0x8000c2c4       0x50 c:/ti/ccsv5/tools/compiler/gcc-arm-none-eabi-4_7-2012q4/bin/../lib/gcc/arm-none-eabi/4.7.3/../../../../arm-none-eabi/lib\librdimon.a(rdimon-syscalls.o)
                0x8000c2c4                _unlink
 .text._gettimeofday
                0x8000c314       0x4c c:/ti/ccsv5/tools/compiler/gcc-arm-none-eabi-4_7-2012q4/bin/../lib/gcc/arm-none-eabi/4.7.3/../../../../arm-none-eabi/lib\librdimon.a(rdimon-syscalls.o)
                0x8000c314                _gettimeofday
 .text._clock   0x8000c360       0x28 c:/ti/ccsv5/tools/compiler/gcc-arm-none-eabi-4_7-2012q4/bin/../lib/gcc/arm-none-eabi/4.7.3/../../../../arm-none-eabi/lib\librdimon.a(rdimon-syscalls.o)
                0x8000c360                _clock
 .text._times   0x8000c388       0x40 c:/ti/ccsv5/tools/compiler/gcc-arm-none-eabi-4_7-2012q4/bin/../lib/gcc/arm-none-eabi/4.7.3/../../../../arm-none-eabi/lib\librdimon.a(rdimon-syscalls.o)
                0x8000c388                _times
 .text._isatty  0x8000c3c8       0x74 c:/ti/ccsv5/tools/compiler/gcc-arm-none-eabi-4_7-2012q4/bin/../lib/gcc/arm-none-eabi/4.7.3/../../../../arm-none-eabi/lib\librdimon.a(rdimon-syscalls.o)
                0x8000c3c8                _isatty
 .text._system  0x8000c43c       0x7c c:/ti/ccsv5/tools/compiler/gcc-arm-none-eabi-4_7-2012q4/bin/../lib/gcc/arm-none-eabi/4.7.3/../../../../arm-none-eabi/lib\librdimon.a(rdimon-syscalls.o)
                0x8000c43c                _system
 .text._rename  0x8000c4b8       0x60 c:/ti/ccsv5/tools/compiler/gcc-arm-none-eabi-4_7-2012q4/bin/../lib/gcc/arm-none-eabi/4.7.3/../../../../arm-none-eabi/lib\librdimon.a(rdimon-syscalls.o)
                0x8000c4b8                _rename
 .text          0x8000c518        0x0 c:/ti/ccsv5/tools/compiler/gcc-arm-none-eabi-4_7-2012q4/bin/../lib/gcc/arm-none-eabi/4.7.3/../../../../arm-none-eabi/lib\librdimon.a(rdimon-_exit.o)
 .text._exit    0x8000c518       0x14 c:/ti/ccsv5/tools/compiler/gcc-arm-none-eabi-4_7-2012q4/bin/../lib/gcc/arm-none-eabi/4.7.3/../../../../arm-none-eabi/lib\librdimon.a(rdimon-_exit.o)
                0x8000c518                _exit
 .text          0x8000c52c        0x0 c:/ti/ccsv5/tools/compiler/gcc-arm-none-eabi-4_7-2012q4/bin/../lib/gcc/arm-none-eabi/4.7.3/../../../../arm-none-eabi/lib\librdimon.a(rdimon-_kill.o)
 .text._kill    0x8000c52c       0x38 c:/ti/ccsv5/tools/compiler/gcc-arm-none-eabi-4_7-2012q4/bin/../lib/gcc/arm-none-eabi/4.7.3/../../../../arm-none-eabi/lib\librdimon.a(rdimon-_kill.o)
                0x8000c52c                _kill
 .text          0x8000c564        0x0 c:/ti/ccsv5/tools/compiler/gcc-arm-none-eabi-4_7-2012q4/bin/../lib/gcc/arm-none-eabi/4.7.3/../../../../arm-none-eabi/lib\libc.a(lib_a-errno.o)
 .text.__errno  0x8000c564       0x10 c:/ti/ccsv5/tools/compiler/gcc-arm-none-eabi-4_7-2012q4/bin/../lib/gcc/arm-none-eabi/4.7.3/../../../../arm-none-eabi/lib\libc.a(lib_a-errno.o)
                0x8000c564                __errno
 .text          0x8000c574        0x0 c:/ti/ccsv5/tools/compiler/gcc-arm-none-eabi-4_7-2012q4/bin/../lib/gcc/arm-none-eabi/4.7.3/crtend.o
 .text          0x8000c574        0x0 c:/ti/ccsv5/tools/compiler/gcc-arm-none-eabi-4_7-2012q4/bin/../lib/gcc/arm-none-eabi/4.7.3/crtn.o
 *(.init)
 .init          0x8000c574        0xc c:/ti/ccsv5/tools/compiler/gcc-arm-none-eabi-4_7-2012q4/bin/../lib/gcc/arm-none-eabi/4.7.3/crti.o
                0x8000c574                _init
 .init          0x8000c580        0xc c:/ti/ccsv5/tools/compiler/gcc-arm-none-eabi-4_7-2012q4/bin/../lib/gcc/arm-none-eabi/4.7.3/crtn.o
 *(.fini)
 .fini          0x8000c58c        0xc c:/ti/ccsv5/tools/compiler/gcc-arm-none-eabi-4_7-2012q4/bin/../lib/gcc/arm-none-eabi/4.7.3/crti.o
                0x8000c58c                _fini
 .fini          0x8000c598        0xc c:/ti/ccsv5/tools/compiler/gcc-arm-none-eabi-4_7-2012q4/bin/../lib/gcc/arm-none-eabi/4.7.3/crtn.o
 *crtbegin.o(.ctors)
 *crtbegin?.o(.ctors)
 *(EXCLUDE_FILE(*crtend.o *crtend?.o) .ctors)
 *(SORT(.ctors.*))
 *(.ctors)
 *crtbegin.o(.dtors)
 *crtbegin?.o(.dtors)
 *(EXCLUDE_FILE(*crtend.o *crtend?.o) .dtors)
 *(SORT(.dtors.*))
 *(.dtors)
 *(.rodata*)
 .rodata.str1.4
                0x8000c5a4       0x9a ./main.o
                                 0x9c (size before relaxing)
 *fill*         0x8000c63e        0x2 00
 .rodata.str1.4
                0x8000c640        0x2 c:/ti/ccsv5/tools/compiler/gcc-arm-none-eabi-4_7-2012q4/bin/../lib/gcc/arm-none-eabi/4.7.3/../../../../arm-none-eabi/lib\libc.a(lib_a-impure.o)
                                  0x4 (size before relaxing)
 *fill*         0x8000c642        0x2 00
 .rodata._global_impure_ptr
                0x8000c644        0x4 c:/ti/ccsv5/tools/compiler/gcc-arm-none-eabi-4_7-2012q4/bin/../lib/gcc/arm-none-eabi/4.7.3/../../../../arm-none-eabi/lib\libc.a(lib_a-impure.o)
                0x8000c644                _global_impure_ptr
 .rodata.str1.4
                0x8000c648        0x2 c:/ti/ccsv5/tools/compiler/gcc-arm-none-eabi-4_7-2012q4/bin/../lib/gcc/arm-none-eabi/4.7.3/../../../../arm-none-eabi/lib\libc.a(lib_a-puts.o)
                                  0x4 (size before relaxing)
 *fill*         0x8000c64a        0x2 00
 .rodata.blanks.6735
                0x8000c64c       0x10 c:/ti/ccsv5/tools/compiler/gcc-arm-none-eabi-4_7-2012q4/bin/../lib/gcc/arm-none-eabi/4.7.3/../../../../arm-none-eabi/lib\libc.a(lib_a-vfprintf.o)
 .rodata.str1.4
                0x8000c65c       0x42 c:/ti/ccsv5/tools/compiler/gcc-arm-none-eabi-4_7-2012q4/bin/../lib/gcc/arm-none-eabi/4.7.3/../../../../arm-none-eabi/lib\libc.a(lib_a-vfprintf.o)
                                 0x44 (size before relaxing)
 *fill*         0x8000c69e        0x2 00
 .rodata.zeroes.6736
                0x8000c6a0       0x10 c:/ti/ccsv5/tools/compiler/gcc-arm-none-eabi-4_7-2012q4/bin/../lib/gcc/arm-none-eabi/4.7.3/../../../../arm-none-eabi/lib\libc.a(lib_a-vfprintf.o)
 .rodata.str1.4
                0x8000c6b0       0x10 c:/ti/ccsv5/tools/compiler/gcc-arm-none-eabi-4_7-2012q4/bin/../lib/gcc/arm-none-eabi/4.7.3/../../../../arm-none-eabi/lib\libc.a(lib_a-dtoa.o)
                                 0x14 (size before relaxing)
 .rodata.str1.4
                0x8000c6c0        0xa c:/ti/ccsv5/tools/compiler/gcc-arm-none-eabi-4_7-2012q4/bin/../lib/gcc/arm-none-eabi/4.7.3/../../../../arm-none-eabi/lib\libc.a(lib_a-locale.o)
                                 0x14 (size before relaxing)
 *fill*         0x8000c6ca        0x2 00
 .rodata.p05.5242
                0x8000c6cc        0xc c:/ti/ccsv5/tools/compiler/gcc-arm-none-eabi-4_7-2012q4/bin/../lib/gcc/arm-none-eabi/4.7.3/../../../../arm-none-eabi/lib\libc.a(lib_a-mprec.o)
 .rodata.__mprec_tens
                0x8000c6d8       0xc8 c:/ti/ccsv5/tools/compiler/gcc-arm-none-eabi-4_7-2012q4/bin/../lib/gcc/arm-none-eabi/4.7.3/../../../../arm-none-eabi/lib\libc.a(lib_a-mprec.o)
                0x8000c6d8                __mprec_tens
 .rodata.__mprec_bigtens
                0x8000c7a0       0x28 c:/ti/ccsv5/tools/compiler/gcc-arm-none-eabi-4_7-2012q4/bin/../lib/gcc/arm-none-eabi/4.7.3/../../../../arm-none-eabi/lib\libc.a(lib_a-mprec.o)
                0x8000c7a0                __mprec_bigtens
 .rodata.__mprec_tinytens
                0x8000c7c8       0x28 c:/ti/ccsv5/tools/compiler/gcc-arm-none-eabi-4_7-2012q4/bin/../lib/gcc/arm-none-eabi/4.7.3/../../../../arm-none-eabi/lib\libc.a(lib_a-mprec.o)
                0x8000c7c8                __mprec_tinytens
 .rodata.blanks.6678
                0x8000c7f0       0x10 c:/ti/ccsv5/tools/compiler/gcc-arm-none-eabi-4_7-2012q4/bin/../lib/gcc/arm-none-eabi/4.7.3/../../../../arm-none-eabi/lib\libc.a(lib_a-vfiprintf.o)
 .rodata.str1.4
                0x00000000       0x30 c:/ti/ccsv5/tools/compiler/gcc-arm-none-eabi-4_7-2012q4/bin/../lib/gcc/arm-none-eabi/4.7.3/../../../../arm-none-eabi/lib\libc.a(lib_a-vfiprintf.o)
 .rodata.zeroes.6679
                0x8000c800       0x10 c:/ti/ccsv5/tools/compiler/gcc-arm-none-eabi-4_7-2012q4/bin/../lib/gcc/arm-none-eabi/4.7.3/../../../../arm-none-eabi/lib\libc.a(lib_a-vfiprintf.o)
 .rodata.str1.4
                0x8000c810        0x4 c:/ti/ccsv5/tools/compiler/gcc-arm-none-eabi-4_7-2012q4/bin/../lib/gcc/arm-none-eabi/4.7.3/../../../../arm-none-eabi/lib\librdimon.a(rdimon-syscalls.o)
 *(.eh_frame*)
 .eh_frame      0x8000c814        0x0 c:/ti/ccsv5/tools/compiler/gcc-arm-none-eabi-4_7-2012q4/bin/../lib/gcc/arm-none-eabi/4.7.3/crtbegin.o
 .eh_frame      0x8000c814        0x4 c:/ti/ccsv5/tools/compiler/gcc-arm-none-eabi-4_7-2012q4/bin/../lib/gcc/arm-none-eabi/4.7.3/crtend.o

.glue_7         0x8000c818        0x0
 .glue_7        0x00000000        0x0 linker stubs

.glue_7t        0x8000c818        0x0
 .glue_7t       0x00000000        0x0 linker stubs

.vfp11_veneer   0x8000c818        0x0
 .vfp11_veneer  0x00000000        0x0 linker stubs

.v4_bx          0x8000c818        0x0
 .v4_bx         0x00000000        0x0 linker stubs

.iplt           0x8000c818        0x0
 .iplt          0x00000000        0x0 c:/ti/ccsv5/tools/compiler/gcc-arm-none-eabi-4_7-2012q4/bin/../lib/gcc/arm-none-eabi/4.7.3/crtbegin.o

.ARM.extab      0x8000c818        0x0
 *(.ARM.extab* .gnu.linkonce.armextab.*)
 .ARM.extab     0x8000c818        0x0 c:/ti/ccsv5/tools/compiler/gcc-arm-none-eabi-4_7-2012q4/bin/../lib/gcc/arm-none-eabi/4.7.3/../../../../arm-none-eabi/lib/rdimon-crt0.o
 .ARM.extab     0x8000c818        0x0 c:/ti/ccsv5/tools/compiler/gcc-arm-none-eabi-4_7-2012q4/bin/../lib/gcc/arm-none-eabi/4.7.3\libgcc.a(_divdi3.o)
 .ARM.extab     0x8000c818        0x0 c:/ti/ccsv5/tools/compiler/gcc-arm-none-eabi-4_7-2012q4/bin/../lib/gcc/arm-none-eabi/4.7.3\libgcc.a(_udivdi3.o)
                0x8000c818                __exidx_start = .

.ARM.exidx      0x8000c818        0x8
 *(.ARM.exidx* .gnu.linkonce.armexidx.*)
 .ARM.exidx     0x8000c818        0x8 c:/ti/ccsv5/tools/compiler/gcc-arm-none-eabi-4_7-2012q4/bin/../lib/gcc/arm-none-eabi/4.7.3/../../../../arm-none-eabi/lib/rdimon-crt0.o
 .ARM.exidx     0x8000c820        0x0 c:/ti/ccsv5/tools/compiler/gcc-arm-none-eabi-4_7-2012q4/bin/../lib/gcc/arm-none-eabi/4.7.3\libgcc.a(_divdi3.o)
                                  0x8 (size before relaxing)
 .ARM.exidx     0x8000c820        0x0 c:/ti/ccsv5/tools/compiler/gcc-arm-none-eabi-4_7-2012q4/bin/../lib/gcc/arm-none-eabi/4.7.3\libgcc.a(_udivdi3.o)
                                  0x8 (size before relaxing)
                0x8000c820                __exidx_end = .

.rel.dyn        0x8000c820        0x0
 .rel.iplt      0x00000000        0x0 c:/ti/ccsv5/tools/compiler/gcc-arm-none-eabi-4_7-2012q4/bin/../lib/gcc/arm-none-eabi/4.7.3/crtbegin.o

.data           0x8000c820      0x9e8
                0x8000c820                . = ALIGN (0x4)
                0x8000c820                __data_start__ = .
 *(vtable)
 *(.data*)
 .data          0x8000c820        0x0 c:/ti/ccsv5/tools/compiler/gcc-arm-none-eabi-4_7-2012q4/bin/../lib/gcc/arm-none-eabi/4.7.3/crti.o
 .data          0x8000c820        0x4 c:/ti/ccsv5/tools/compiler/gcc-arm-none-eabi-4_7-2012q4/bin/../lib/gcc/arm-none-eabi/4.7.3/crtbegin.o
                0x8000c820                __dso_handle
 .data          0x8000c824      0x110 c:/ti/ccsv5/tools/compiler/gcc-arm-none-eabi-4_7-2012q4/bin/../lib/gcc/arm-none-eabi/4.7.3/../../../../arm-none-eabi/lib/rdimon-crt0.o
                0x8000c82c                __stack_base__
 .data          0x8000c934        0x0 ./common_arm/v7_pmu.o
 .data          0x8000c934        0x0 ./common_arm/utilFxns.o
 .data          0x8000c934        0x0 ./common_arm/arm_utility.o
 .data          0x8000c934        0x0 ./common_arm/arm_cpintc.o
 .data          0x8000c934        0x0 ./common_arm/aintc_inth.o
 .data          0x8000c934        0x4 ./common_arm/GIC_ctl.o
                0x8000c934                glbArmVectID
 .data          0x8000c938        0x0 ./common_arm/Cortex_A_generic_timer.o
 .data          0x8000c938        0x0 ./startup_ARMCA8.o
 .data          0x8000c938        0x4 ./main.o
                0x8000c938                ptrGIC400_Handle
 .data          0x8000c93c        0x0 c:/ti/ccsv5/tools/compiler/gcc-arm-none-eabi-4_7-2012q4/bin/../lib/gcc/arm-none-eabi/4.7.3/../../../../arm-none-eabi/lib\libc.a(lib_a-__atexit.o)
 .data          0x8000c93c        0x0 c:/ti/ccsv5/tools/compiler/gcc-arm-none-eabi-4_7-2012q4/bin/../lib/gcc/arm-none-eabi/4.7.3/../../../../arm-none-eabi/lib\libc.a(lib_a-exit.o)
 .data          0x8000c93c        0x0 c:/ti/ccsv5/tools/compiler/gcc-arm-none-eabi-4_7-2012q4/bin/../lib/gcc/arm-none-eabi/4.7.3/../../../../arm-none-eabi/lib\libc.a(lib_a-fini.o)
 .data          0x8000c93c        0x0 c:/ti/ccsv5/tools/compiler/gcc-arm-none-eabi-4_7-2012q4/bin/../lib/gcc/arm-none-eabi/4.7.3/../../../../arm-none-eabi/lib\libc.a(lib_a-impure.o)
 *fill*         0x8000c93c        0x4 00
 .data.impure_data
                0x8000c940      0x428 c:/ti/ccsv5/tools/compiler/gcc-arm-none-eabi-4_7-2012q4/bin/../lib/gcc/arm-none-eabi/4.7.3/../../../../arm-none-eabi/lib\libc.a(lib_a-impure.o)
 .data._impure_ptr
                0x8000cd68        0x4 c:/ti/ccsv5/tools/compiler/gcc-arm-none-eabi-4_7-2012q4/bin/../lib/gcc/arm-none-eabi/4.7.3/../../../../arm-none-eabi/lib\libc.a(lib_a-impure.o)
                0x8000cd68                _impure_ptr
 .data          0x8000cd6c        0x0 c:/ti/ccsv5/tools/compiler/gcc-arm-none-eabi-4_7-2012q4/bin/../lib/gcc/arm-none-eabi/4.7.3/../../../../arm-none-eabi/lib\libc.a(lib_a-init.o)
 .data          0x8000cd6c        0x0 c:/ti/ccsv5/tools/compiler/gcc-arm-none-eabi-4_7-2012q4/bin/../lib/gcc/arm-none-eabi/4.7.3/../../../../arm-none-eabi/lib\libc.a(lib_a-memset.o)
 .data          0x8000cd6c        0x0 c:/ti/ccsv5/tools/compiler/gcc-arm-none-eabi-4_7-2012q4/bin/../lib/gcc/arm-none-eabi/4.7.3/../../../../arm-none-eabi/lib\libc.a(lib_a-printf.o)
 .data          0x8000cd6c        0x0 c:/ti/ccsv5/tools/compiler/gcc-arm-none-eabi-4_7-2012q4/bin/../lib/gcc/arm-none-eabi/4.7.3/../../../../arm-none-eabi/lib\libc.a(lib_a-puts.o)
 .data          0x8000cd6c        0x0 c:/ti/ccsv5/tools/compiler/gcc-arm-none-eabi-4_7-2012q4/bin/../lib/gcc/arm-none-eabi/4.7.3/../../../../arm-none-eabi/lib\libc.a(lib_a-strlen.o)
 .data          0x8000cd6c        0x0 c:/ti/ccsv5/tools/compiler/gcc-arm-none-eabi-4_7-2012q4/bin/../lib/gcc/arm-none-eabi/4.7.3/../../../../arm-none-eabi/lib\libc.a(lib_a-vfprintf.o)
 .data          0x8000cd6c        0x0 c:/ti/ccsv5/tools/compiler/gcc-arm-none-eabi-4_7-2012q4/bin/../lib/gcc/arm-none-eabi/4.7.3/../../../../arm-none-eabi/lib\libc.a(lib_a-wsetup.o)
 .data          0x8000cd6c        0x0 c:/ti/ccsv5/tools/compiler/gcc-arm-none-eabi-4_7-2012q4/bin/../lib/gcc/arm-none-eabi/4.7.3/../../../../arm-none-eabi/lib\libc.a(lib_a-__call_atexit.o)
 .data          0x8000cd6c        0x0 c:/ti/ccsv5/tools/compiler/gcc-arm-none-eabi-4_7-2012q4/bin/../lib/gcc/arm-none-eabi/4.7.3/../../../../arm-none-eabi/lib\libc.a(lib_a-atexit.o)
 .data          0x8000cd6c        0x0 c:/ti/ccsv5/tools/compiler/gcc-arm-none-eabi-4_7-2012q4/bin/../lib/gcc/arm-none-eabi/4.7.3/../../../../arm-none-eabi/lib\libc.a(lib_a-dtoa.o)
 .data          0x8000cd6c        0x0 c:/ti/ccsv5/tools/compiler/gcc-arm-none-eabi-4_7-2012q4/bin/../lib/gcc/arm-none-eabi/4.7.3/../../../../arm-none-eabi/lib\libc.a(lib_a-fflush.o)
 .data          0x8000cd6c        0x0 c:/ti/ccsv5/tools/compiler/gcc-arm-none-eabi-4_7-2012q4/bin/../lib/gcc/arm-none-eabi/4.7.3/../../../../arm-none-eabi/lib\libc.a(lib_a-findfp.o)
 .data          0x8000cd6c        0x0 c:/ti/ccsv5/tools/compiler/gcc-arm-none-eabi-4_7-2012q4/bin/../lib/gcc/arm-none-eabi/4.7.3/../../../../arm-none-eabi/lib\libc.a(lib_a-freer.o)
 .data          0x8000cd6c        0x0 c:/ti/ccsv5/tools/compiler/gcc-arm-none-eabi-4_7-2012q4/bin/../lib/gcc/arm-none-eabi/4.7.3/../../../../arm-none-eabi/lib\libc.a(lib_a-fvwrite.o)
 .data          0x8000cd6c        0x0 c:/ti/ccsv5/tools/compiler/gcc-arm-none-eabi-4_7-2012q4/bin/../lib/gcc/arm-none-eabi/4.7.3/../../../../arm-none-eabi/lib\libc.a(lib_a-fwalk.o)
 .data          0x8000cd6c        0x0 c:/ti/ccsv5/tools/compiler/gcc-arm-none-eabi-4_7-2012q4/bin/../lib/gcc/arm-none-eabi/4.7.3/../../../../arm-none-eabi/lib\libc.a(lib_a-locale.o)
 .data.lc_message_charset
                0x8000cd6c       0x20 c:/ti/ccsv5/tools/compiler/gcc-arm-none-eabi-4_7-2012q4/bin/../lib/gcc/arm-none-eabi/4.7.3/../../../../arm-none-eabi/lib\libc.a(lib_a-locale.o)
 .data.lconv    0x8000cd8c       0x38 c:/ti/ccsv5/tools/compiler/gcc-arm-none-eabi-4_7-2012q4/bin/../lib/gcc/arm-none-eabi/4.7.3/../../../../arm-none-eabi/lib\libc.a(lib_a-locale.o)
 .data.lc_ctype_charset
                0x8000cdc4       0x20 c:/ti/ccsv5/tools/compiler/gcc-arm-none-eabi-4_7-2012q4/bin/../lib/gcc/arm-none-eabi/4.7.3/../../../../arm-none-eabi/lib\libc.a(lib_a-locale.o)
 .data.__mb_cur_max
                0x8000cde4        0x4 c:/ti/ccsv5/tools/compiler/gcc-arm-none-eabi-4_7-2012q4/bin/../lib/gcc/arm-none-eabi/4.7.3/../../../../arm-none-eabi/lib\libc.a(lib_a-locale.o)
                0x8000cde4                __mb_cur_max
 .data          0x8000cde8        0x0 c:/ti/ccsv5/tools/compiler/gcc-arm-none-eabi-4_7-2012q4/bin/../lib/gcc/arm-none-eabi/4.7.3/../../../../arm-none-eabi/lib\libc.a(lib_a-makebuf.o)
 .data          0x8000cde8        0x0 c:/ti/ccsv5/tools/compiler/gcc-arm-none-eabi-4_7-2012q4/bin/../lib/gcc/arm-none-eabi/4.7.3/../../../../arm-none-eabi/lib\libc.a(lib_a-mallocr.o)
 .data.__malloc_av_
                0x8000cde8      0x408 c:/ti/ccsv5/tools/compiler/gcc-arm-none-eabi-4_7-2012q4/bin/../lib/gcc/arm-none-eabi/4.7.3/../../../../arm-none-eabi/lib\libc.a(lib_a-mallocr.o)
                0x8000cde8                __malloc_av_
 .data.__malloc_trim_threshold
                0x8000d1f0        0x4 c:/ti/ccsv5/tools/compiler/gcc-arm-none-eabi-4_7-2012q4/bin/../lib/gcc/arm-none-eabi/4.7.3/../../../../arm-none-eabi/lib\libc.a(lib_a-mallocr.o)
                0x8000d1f0                __malloc_trim_threshold
 .data.__malloc_sbrk_base
                0x8000d1f4        0x4 c:/ti/ccsv5/tools/compiler/gcc-arm-none-eabi-4_7-2012q4/bin/../lib/gcc/arm-none-eabi/4.7.3/../../../../arm-none-eabi/lib\libc.a(lib_a-mallocr.o)
                0x8000d1f4                __malloc_sbrk_base
 .data          0x8000d1f8        0x0 c:/ti/ccsv5/tools/compiler/gcc-arm-none-eabi-4_7-2012q4/bin/../lib/gcc/arm-none-eabi/4.7.3/../../../../arm-none-eabi/lib\libc.a(lib_a-memchr.o)
 .data          0x8000d1f8        0x0 c:/ti/ccsv5/tools/compiler/gcc-arm-none-eabi-4_7-2012q4/bin/../lib/gcc/arm-none-eabi/4.7.3/../../../../arm-none-eabi/lib\libc.a(lib_a-memcpy.o)
 .data          0x8000d1f8        0x0 c:/ti/ccsv5/tools/compiler/gcc-arm-none-eabi-4_7-2012q4/bin/../lib/gcc/arm-none-eabi/4.7.3/../../../../arm-none-eabi/lib\libc.a(lib_a-memmove.o)
 .data          0x8000d1f8        0x0 c:/ti/ccsv5/tools/compiler/gcc-arm-none-eabi-4_7-2012q4/bin/../lib/gcc/arm-none-eabi/4.7.3/../../../../arm-none-eabi/lib\libc.a(lib_a-mlock.o)
 .data          0x8000d1f8        0x0 c:/ti/ccsv5/tools/compiler/gcc-arm-none-eabi-4_7-2012q4/bin/../lib/gcc/arm-none-eabi/4.7.3/../../../../arm-none-eabi/lib\libc.a(lib_a-mprec.o)
 .data          0x8000d1f8        0x0 c:/ti/ccsv5/tools/compiler/gcc-arm-none-eabi-4_7-2012q4/bin/../lib/gcc/arm-none-eabi/4.7.3/../../../../arm-none-eabi/lib\libc.a(lib_a-reallocr.o)
 .data          0x8000d1f8        0x0 c:/ti/ccsv5/tools/compiler/gcc-arm-none-eabi-4_7-2012q4/bin/../lib/gcc/arm-none-eabi/4.7.3/../../../../arm-none-eabi/lib\libc.a(lib_a-s_fpclassify.o)
 .data          0x8000d1f8        0x0 c:/ti/ccsv5/tools/compiler/gcc-arm-none-eabi-4_7-2012q4/bin/../lib/gcc/arm-none-eabi/4.7.3/../../../../arm-none-eabi/lib\libc.a(lib_a-sbrkr.o)
 .data          0x8000d1f8        0x0 c:/ti/ccsv5/tools/compiler/gcc-arm-none-eabi-4_7-2012q4/bin/../lib/gcc/arm-none-eabi/4.7.3/../../../../arm-none-eabi/lib\libc.a(lib_a-stdio.o)
 .data          0x8000d1f8        0x0 c:/ti/ccsv5/tools/compiler/gcc-arm-none-eabi-4_7-2012q4/bin/../lib/gcc/arm-none-eabi/4.7.3/../../../../arm-none-eabi/lib\libc.a(lib_a-strcmp.o)
 .data          0x8000d1f8        0x0 c:/ti/ccsv5/tools/compiler/gcc-arm-none-eabi-4_7-2012q4/bin/../lib/gcc/arm-none-eabi/4.7.3/../../../../arm-none-eabi/lib\libc.a(lib_a-vfiprintf.o)
 .data          0x8000d1f8        0x0 c:/ti/ccsv5/tools/compiler/gcc-arm-none-eabi-4_7-2012q4/bin/../lib/gcc/arm-none-eabi/4.7.3/../../../../arm-none-eabi/lib\libc.a(lib_a-writer.o)
 .data          0x8000d1f8        0x0 c:/ti/ccsv5/tools/compiler/gcc-arm-none-eabi-4_7-2012q4/bin/../lib/gcc/arm-none-eabi/4.7.3/../../../../arm-none-eabi/lib\libc.a(lib_a-callocr.o)
 .data          0x8000d1f8        0x0 c:/ti/ccsv5/tools/compiler/gcc-arm-none-eabi-4_7-2012q4/bin/../lib/gcc/arm-none-eabi/4.7.3/../../../../arm-none-eabi/lib\libc.a(lib_a-closer.o)
 .data          0x8000d1f8        0x0 c:/ti/ccsv5/tools/compiler/gcc-arm-none-eabi-4_7-2012q4/bin/../lib/gcc/arm-none-eabi/4.7.3/../../../../arm-none-eabi/lib\libc.a(lib_a-fclose.o)
 .data          0x8000d1f8        0x0 c:/ti/ccsv5/tools/compiler/gcc-arm-none-eabi-4_7-2012q4/bin/../lib/gcc/arm-none-eabi/4.7.3/../../../../arm-none-eabi/lib\libc.a(lib_a-fputwc.o)
 .data          0x8000d1f8        0x0 c:/ti/ccsv5/tools/compiler/gcc-arm-none-eabi-4_7-2012q4/bin/../lib/gcc/arm-none-eabi/4.7.3/../../../../arm-none-eabi/lib\libc.a(lib_a-fstatr.o)
 .data          0x8000d1f8        0x0 c:/ti/ccsv5/tools/compiler/gcc-arm-none-eabi-4_7-2012q4/bin/../lib/gcc/arm-none-eabi/4.7.3/../../../../arm-none-eabi/lib\libc.a(lib_a-isattyr.o)
 .data          0x8000d1f8        0x0 c:/ti/ccsv5/tools/compiler/gcc-arm-none-eabi-4_7-2012q4/bin/../lib/gcc/arm-none-eabi/4.7.3/../../../../arm-none-eabi/lib\libc.a(lib_a-lseekr.o)
 .data          0x8000d1f8        0x0 c:/ti/ccsv5/tools/compiler/gcc-arm-none-eabi-4_7-2012q4/bin/../lib/gcc/arm-none-eabi/4.7.3/../../../../arm-none-eabi/lib\libc.a(lib_a-readr.o)
 .data          0x8000d1f8        0x0 c:/ti/ccsv5/tools/compiler/gcc-arm-none-eabi-4_7-2012q4/bin/../lib/gcc/arm-none-eabi/4.7.3/../../../../arm-none-eabi/lib\libc.a(lib_a-reent.o)
 .data          0x8000d1f8        0x0 c:/ti/ccsv5/tools/compiler/gcc-arm-none-eabi-4_7-2012q4/bin/../lib/gcc/arm-none-eabi/4.7.3/../../../../arm-none-eabi/lib\libc.a(lib_a-wbuf.o)
 .data          0x8000d1f8        0x0 c:/ti/ccsv5/tools/compiler/gcc-arm-none-eabi-4_7-2012q4/bin/../lib/gcc/arm-none-eabi/4.7.3/../../../../arm-none-eabi/lib\libc.a(lib_a-wcrtomb.o)
 .data          0x8000d1f8        0x0 c:/ti/ccsv5/tools/compiler/gcc-arm-none-eabi-4_7-2012q4/bin/../lib/gcc/arm-none-eabi/4.7.3/../../../../arm-none-eabi/lib\libc.a(lib_a-wctomb_r.o)
 .data.__wctomb
                0x8000d1f8        0x4 c:/ti/ccsv5/tools/compiler/gcc-arm-none-eabi-4_7-2012q4/bin/../lib/gcc/arm-none-eabi/4.7.3/../../../../arm-none-eabi/lib\libc.a(lib_a-wctomb_r.o)
                0x8000d1f8                __wctomb
 .data          0x8000d1fc        0x0 c:/ti/ccsv5/tools/compiler/gcc-arm-none-eabi-4_7-2012q4/bin/../lib/gcc/arm-none-eabi/4.7.3\libgcc.a(_udivsi3.o)
 .data          0x8000d1fc        0x0 c:/ti/ccsv5/tools/compiler/gcc-arm-none-eabi-4_7-2012q4/bin/../lib/gcc/arm-none-eabi/4.7.3\libgcc.a(_dvmd_tls.o)
 .data          0x8000d1fc        0x0 c:/ti/ccsv5/tools/compiler/gcc-arm-none-eabi-4_7-2012q4/bin/../lib/gcc/arm-none-eabi/4.7.3\libgcc.a(_arm_addsubdf3.o)
 .data          0x8000d1fc        0x0 c:/ti/ccsv5/tools/compiler/gcc-arm-none-eabi-4_7-2012q4/bin/../lib/gcc/arm-none-eabi/4.7.3\libgcc.a(_arm_muldivdf3.o)
 .data          0x8000d1fc        0x0 c:/ti/ccsv5/tools/compiler/gcc-arm-none-eabi-4_7-2012q4/bin/../lib/gcc/arm-none-eabi/4.7.3\libgcc.a(_arm_cmpdf2.o)
 .data          0x8000d1fc        0x0 c:/ti/ccsv5/tools/compiler/gcc-arm-none-eabi-4_7-2012q4/bin/../lib/gcc/arm-none-eabi/4.7.3\libgcc.a(_arm_fixdfsi.o)
 .data          0x8000d1fc        0x0 c:/ti/ccsv5/tools/compiler/gcc-arm-none-eabi-4_7-2012q4/bin/../lib/gcc/arm-none-eabi/4.7.3\libgcc.a(_aeabi_uldivmod.o)
 .data          0x8000d1fc        0x0 c:/ti/ccsv5/tools/compiler/gcc-arm-none-eabi-4_7-2012q4/bin/../lib/gcc/arm-none-eabi/4.7.3\libgcc.a(bpabi.o)
 .data          0x8000d1fc        0x0 c:/ti/ccsv5/tools/compiler/gcc-arm-none-eabi-4_7-2012q4/bin/../lib/gcc/arm-none-eabi/4.7.3\libgcc.a(_divdi3.o)
 .data          0x8000d1fc        0x0 c:/ti/ccsv5/tools/compiler/gcc-arm-none-eabi-4_7-2012q4/bin/../lib/gcc/arm-none-eabi/4.7.3\libgcc.a(_udivdi3.o)
 .data          0x8000d1fc        0x0 c:/ti/ccsv5/tools/compiler/gcc-arm-none-eabi-4_7-2012q4/bin/../lib/gcc/arm-none-eabi/4.7.3\libgcc.a(_clzsi2.o)
 .data          0x8000d1fc        0x0 c:/ti/ccsv5/tools/compiler/gcc-arm-none-eabi-4_7-2012q4/bin/../lib/gcc/arm-none-eabi/4.7.3/../../../../arm-none-eabi/lib\librdimon.a(rdimon-syscalls.o)
 .data          0x8000d1fc        0x0 c:/ti/ccsv5/tools/compiler/gcc-arm-none-eabi-4_7-2012q4/bin/../lib/gcc/arm-none-eabi/4.7.3/../../../../arm-none-eabi/lib\librdimon.a(rdimon-_exit.o)
 .data          0x8000d1fc        0x0 c:/ti/ccsv5/tools/compiler/gcc-arm-none-eabi-4_7-2012q4/bin/../lib/gcc/arm-none-eabi/4.7.3/../../../../arm-none-eabi/lib\librdimon.a(rdimon-_kill.o)
 .data          0x8000d1fc        0x0 c:/ti/ccsv5/tools/compiler/gcc-arm-none-eabi-4_7-2012q4/bin/../lib/gcc/arm-none-eabi/4.7.3/../../../../arm-none-eabi/lib\libc.a(lib_a-errno.o)
 .data          0x8000d1fc        0x0 c:/ti/ccsv5/tools/compiler/gcc-arm-none-eabi-4_7-2012q4/bin/../lib/gcc/arm-none-eabi/4.7.3/crtend.o
 .data          0x8000d1fc        0x0 c:/ti/ccsv5/tools/compiler/gcc-arm-none-eabi-4_7-2012q4/bin/../lib/gcc/arm-none-eabi/4.7.3/crtn.o
                0x8000d1fc                . = ALIGN (0x4)
                0x8000d1fc                PROVIDE (__preinit_array_start, .)
 *(.preinit_array)
                0x8000d1fc                PROVIDE (__preinit_array_end, .)
                0x8000d1fc                . = ALIGN (0x4)
                0x8000d1fc                PROVIDE (__init_array_start, .)
 *(SORT(.init_array.*))
 .init_array.00000
                0x8000d1fc        0x4 c:/ti/ccsv5/tools/compiler/gcc-arm-none-eabi-4_7-2012q4/bin/../lib/gcc/arm-none-eabi/4.7.3/../../../../arm-none-eabi/lib\libc.a(lib_a-__call_atexit.o)
 *(.init_array)
 .init_array    0x8000d200        0x4 c:/ti/ccsv5/tools/compiler/gcc-arm-none-eabi-4_7-2012q4/bin/../lib/gcc/arm-none-eabi/4.7.3/crtbegin.o
                0x8000d204                PROVIDE (__init_array_end, .)
                0x8000d204                . = ALIGN (0x4)
                0x8000d204                PROVIDE (__fini_array_start, .)
 *(SORT(.fini_array.*))
 *(.fini_array)
 .fini_array    0x8000d204        0x4 c:/ti/ccsv5/tools/compiler/gcc-arm-none-eabi-4_7-2012q4/bin/../lib/gcc/arm-none-eabi/4.7.3/crtbegin.o
                0x8000d208                PROVIDE (__fini_array_end, .)
                0x8000d208                . = ALIGN (0x4)
                0x8000d208                __data_end__ = .

.jcr            0x8000d208        0x4
 .jcr           0x8000d208        0x0 c:/ti/ccsv5/tools/compiler/gcc-arm-none-eabi-4_7-2012q4/bin/../lib/gcc/arm-none-eabi/4.7.3/crtbegin.o
 .jcr           0x8000d208        0x4 c:/ti/ccsv5/tools/compiler/gcc-arm-none-eabi-4_7-2012q4/bin/../lib/gcc/arm-none-eabi/4.7.3/crtend.o

.igot.plt       0x8000d20c        0x0
 .igot.plt      0x00000000        0x0 c:/ti/ccsv5/tools/compiler/gcc-arm-none-eabi-4_7-2012q4/bin/../lib/gcc/arm-none-eabi/4.7.3/crtbegin.o

.bss            0x8000d20c     0x111c
                0x8000d20c                . = ALIGN (0x4)
                0x8000d20c                __bss_start__ = .
 *(.bss*)
 .bss           0x8000d20c        0x0 c:/ti/ccsv5/tools/compiler/gcc-arm-none-eabi-4_7-2012q4/bin/../lib/gcc/arm-none-eabi/4.7.3/crti.o
 .bss           0x8000d20c       0x1c c:/ti/ccsv5/tools/compiler/gcc-arm-none-eabi-4_7-2012q4/bin/../lib/gcc/arm-none-eabi/4.7.3/crtbegin.o
 .bss           0x8000d228        0x0 c:/ti/ccsv5/tools/compiler/gcc-arm-none-eabi-4_7-2012q4/bin/../lib/gcc/arm-none-eabi/4.7.3/../../../../arm-none-eabi/lib/rdimon-crt0.o
 .bss           0x8000d228        0x0 ./common_arm/v7_pmu.o
 .bss           0x8000d228        0x0 ./common_arm/utilFxns.o
 .bss           0x8000d228        0x0 ./common_arm/arm_utility.o
 .bss           0x8000d228        0x4 ./common_arm/arm_cpintc.o
 .bss           0x8000d22c     0x1004 ./common_arm/aintc_inth.o
 .bss           0x8000e230        0x0 ./common_arm/GIC_ctl.o
 .bss           0x8000e230        0x0 ./common_arm/Cortex_A_generic_timer.o
 .bss           0x8000e230        0x0 ./startup_ARMCA8.o
 .bss           0x8000e230        0x4 ./main.o
                0x8000e230                uiTick
 .bss           0x8000e234        0x0 c:/ti/ccsv5/tools/compiler/gcc-arm-none-eabi-4_7-2012q4/bin/../lib/gcc/arm-none-eabi/4.7.3/../../../../arm-none-eabi/lib\libc.a(lib_a-__atexit.o)
 .bss           0x8000e234        0x0 c:/ti/ccsv5/tools/compiler/gcc-arm-none-eabi-4_7-2012q4/bin/../lib/gcc/arm-none-eabi/4.7.3/../../../../arm-none-eabi/lib\libc.a(lib_a-exit.o)
 .bss           0x8000e234        0x0 c:/ti/ccsv5/tools/compiler/gcc-arm-none-eabi-4_7-2012q4/bin/../lib/gcc/arm-none-eabi/4.7.3/../../../../arm-none-eabi/lib\libc.a(lib_a-fini.o)
 .bss           0x8000e234        0x0 c:/ti/ccsv5/tools/compiler/gcc-arm-none-eabi-4_7-2012q4/bin/../lib/gcc/arm-none-eabi/4.7.3/../../../../arm-none-eabi/lib\libc.a(lib_a-impure.o)
 .bss           0x8000e234        0x0 c:/ti/ccsv5/tools/compiler/gcc-arm-none-eabi-4_7-2012q4/bin/../lib/gcc/arm-none-eabi/4.7.3/../../../../arm-none-eabi/lib\libc.a(lib_a-init.o)
 .bss           0x8000e234        0x0 c:/ti/ccsv5/tools/compiler/gcc-arm-none-eabi-4_7-2012q4/bin/../lib/gcc/arm-none-eabi/4.7.3/../../../../arm-none-eabi/lib\libc.a(lib_a-memset.o)
 .bss           0x8000e234        0x0 c:/ti/ccsv5/tools/compiler/gcc-arm-none-eabi-4_7-2012q4/bin/../lib/gcc/arm-none-eabi/4.7.3/../../../../arm-none-eabi/lib\libc.a(lib_a-printf.o)
 .bss           0x8000e234        0x0 c:/ti/ccsv5/tools/compiler/gcc-arm-none-eabi-4_7-2012q4/bin/../lib/gcc/arm-none-eabi/4.7.3/../../../../arm-none-eabi/lib\libc.a(lib_a-puts.o)
 .bss           0x8000e234        0x0 c:/ti/ccsv5/tools/compiler/gcc-arm-none-eabi-4_7-2012q4/bin/../lib/gcc/arm-none-eabi/4.7.3/../../../../arm-none-eabi/lib\libc.a(lib_a-strlen.o)
 .bss           0x8000e234        0x0 c:/ti/ccsv5/tools/compiler/gcc-arm-none-eabi-4_7-2012q4/bin/../lib/gcc/arm-none-eabi/4.7.3/../../../../arm-none-eabi/lib\libc.a(lib_a-vfprintf.o)
 .bss           0x8000e234        0x0 c:/ti/ccsv5/tools/compiler/gcc-arm-none-eabi-4_7-2012q4/bin/../lib/gcc/arm-none-eabi/4.7.3/../../../../arm-none-eabi/lib\libc.a(lib_a-wsetup.o)
 .bss           0x8000e234        0x0 c:/ti/ccsv5/tools/compiler/gcc-arm-none-eabi-4_7-2012q4/bin/../lib/gcc/arm-none-eabi/4.7.3/../../../../arm-none-eabi/lib\libc.a(lib_a-__call_atexit.o)
 .bss           0x8000e234        0x0 c:/ti/ccsv5/tools/compiler/gcc-arm-none-eabi-4_7-2012q4/bin/../lib/gcc/arm-none-eabi/4.7.3/../../../../arm-none-eabi/lib\libc.a(lib_a-atexit.o)
 .bss           0x8000e234        0x0 c:/ti/ccsv5/tools/compiler/gcc-arm-none-eabi-4_7-2012q4/bin/../lib/gcc/arm-none-eabi/4.7.3/../../../../arm-none-eabi/lib\libc.a(lib_a-dtoa.o)
 .bss           0x8000e234        0x0 c:/ti/ccsv5/tools/compiler/gcc-arm-none-eabi-4_7-2012q4/bin/../lib/gcc/arm-none-eabi/4.7.3/../../../../arm-none-eabi/lib\libc.a(lib_a-fflush.o)
 .bss           0x8000e234        0x0 c:/ti/ccsv5/tools/compiler/gcc-arm-none-eabi-4_7-2012q4/bin/../lib/gcc/arm-none-eabi/4.7.3/../../../../arm-none-eabi/lib\libc.a(lib_a-findfp.o)
 .bss           0x8000e234        0x0 c:/ti/ccsv5/tools/compiler/gcc-arm-none-eabi-4_7-2012q4/bin/../lib/gcc/arm-none-eabi/4.7.3/../../../../arm-none-eabi/lib\libc.a(lib_a-freer.o)
 .bss           0x8000e234        0x0 c:/ti/ccsv5/tools/compiler/gcc-arm-none-eabi-4_7-2012q4/bin/../lib/gcc/arm-none-eabi/4.7.3/../../../../arm-none-eabi/lib\libc.a(lib_a-fvwrite.o)
 .bss           0x8000e234        0x0 c:/ti/ccsv5/tools/compiler/gcc-arm-none-eabi-4_7-2012q4/bin/../lib/gcc/arm-none-eabi/4.7.3/../../../../arm-none-eabi/lib\libc.a(lib_a-fwalk.o)
 .bss           0x8000e234        0x0 c:/ti/ccsv5/tools/compiler/gcc-arm-none-eabi-4_7-2012q4/bin/../lib/gcc/arm-none-eabi/4.7.3/../../../../arm-none-eabi/lib\libc.a(lib_a-locale.o)
 .bss._PathLocale
                0x8000e234        0x4 c:/ti/ccsv5/tools/compiler/gcc-arm-none-eabi-4_7-2012q4/bin/../lib/gcc/arm-none-eabi/4.7.3/../../../../arm-none-eabi/lib\libc.a(lib_a-locale.o)
                0x8000e234                _PathLocale
 .bss.__nlocale_changed
                0x8000e238        0x4 c:/ti/ccsv5/tools/compiler/gcc-arm-none-eabi-4_7-2012q4/bin/../lib/gcc/arm-none-eabi/4.7.3/../../../../arm-none-eabi/lib\libc.a(lib_a-locale.o)
                0x8000e238                __nlocale_changed
 .bss.__mlocale_changed
                0x8000e23c        0x4 c:/ti/ccsv5/tools/compiler/gcc-arm-none-eabi-4_7-2012q4/bin/../lib/gcc/arm-none-eabi/4.7.3/../../../../arm-none-eabi/lib\libc.a(lib_a-locale.o)
                0x8000e23c                __mlocale_changed
 .bss           0x8000e240        0x0 c:/ti/ccsv5/tools/compiler/gcc-arm-none-eabi-4_7-2012q4/bin/../lib/gcc/arm-none-eabi/4.7.3/../../../../arm-none-eabi/lib\libc.a(lib_a-makebuf.o)
 .bss           0x8000e240        0x0 c:/ti/ccsv5/tools/compiler/gcc-arm-none-eabi-4_7-2012q4/bin/../lib/gcc/arm-none-eabi/4.7.3/../../../../arm-none-eabi/lib\libc.a(lib_a-mallocr.o)
 .bss.__malloc_max_total_mem
                0x8000e240        0x4 c:/ti/ccsv5/tools/compiler/gcc-arm-none-eabi-4_7-2012q4/bin/../lib/gcc/arm-none-eabi/4.7.3/../../../../arm-none-eabi/lib\libc.a(lib_a-mallocr.o)
                0x8000e240                __malloc_max_total_mem
 .bss.__malloc_max_sbrked_mem
                0x8000e244        0x4 c:/ti/ccsv5/tools/compiler/gcc-arm-none-eabi-4_7-2012q4/bin/../lib/gcc/arm-none-eabi/4.7.3/../../../../arm-none-eabi/lib\libc.a(lib_a-mallocr.o)
                0x8000e244                __malloc_max_sbrked_mem
 .bss.__malloc_top_pad
                0x8000e248        0x4 c:/ti/ccsv5/tools/compiler/gcc-arm-none-eabi-4_7-2012q4/bin/../lib/gcc/arm-none-eabi/4.7.3/../../../../arm-none-eabi/lib\libc.a(lib_a-mallocr.o)
                0x8000e248                __malloc_top_pad
 .bss.__malloc_current_mallinfo
                0x8000e24c       0x28 c:/ti/ccsv5/tools/compiler/gcc-arm-none-eabi-4_7-2012q4/bin/../lib/gcc/arm-none-eabi/4.7.3/../../../../arm-none-eabi/lib\libc.a(lib_a-mallocr.o)
                0x8000e24c                __malloc_current_mallinfo
 .bss           0x8000e274        0x0 c:/ti/ccsv5/tools/compiler/gcc-arm-none-eabi-4_7-2012q4/bin/../lib/gcc/arm-none-eabi/4.7.3/../../../../arm-none-eabi/lib\libc.a(lib_a-memchr.o)
 .bss           0x8000e274        0x0 c:/ti/ccsv5/tools/compiler/gcc-arm-none-eabi-4_7-2012q4/bin/../lib/gcc/arm-none-eabi/4.7.3/../../../../arm-none-eabi/lib\libc.a(lib_a-memcpy.o)
 .bss           0x8000e274        0x0 c:/ti/ccsv5/tools/compiler/gcc-arm-none-eabi-4_7-2012q4/bin/../lib/gcc/arm-none-eabi/4.7.3/../../../../arm-none-eabi/lib\libc.a(lib_a-memmove.o)
 .bss           0x8000e274        0x0 c:/ti/ccsv5/tools/compiler/gcc-arm-none-eabi-4_7-2012q4/bin/../lib/gcc/arm-none-eabi/4.7.3/../../../../arm-none-eabi/lib\libc.a(lib_a-mlock.o)
 .bss           0x8000e274        0x0 c:/ti/ccsv5/tools/compiler/gcc-arm-none-eabi-4_7-2012q4/bin/../lib/gcc/arm-none-eabi/4.7.3/../../../../arm-none-eabi/lib\libc.a(lib_a-mprec.o)
 .bss           0x8000e274        0x0 c:/ti/ccsv5/tools/compiler/gcc-arm-none-eabi-4_7-2012q4/bin/../lib/gcc/arm-none-eabi/4.7.3/../../../../arm-none-eabi/lib\libc.a(lib_a-reallocr.o)
 .bss           0x8000e274        0x0 c:/ti/ccsv5/tools/compiler/gcc-arm-none-eabi-4_7-2012q4/bin/../lib/gcc/arm-none-eabi/4.7.3/../../../../arm-none-eabi/lib\libc.a(lib_a-s_fpclassify.o)
 .bss           0x8000e274        0x0 c:/ti/ccsv5/tools/compiler/gcc-arm-none-eabi-4_7-2012q4/bin/../lib/gcc/arm-none-eabi/4.7.3/../../../../arm-none-eabi/lib\libc.a(lib_a-sbrkr.o)
 .bss           0x8000e274        0x0 c:/ti/ccsv5/tools/compiler/gcc-arm-none-eabi-4_7-2012q4/bin/../lib/gcc/arm-none-eabi/4.7.3/../../../../arm-none-eabi/lib\libc.a(lib_a-stdio.o)
 .bss           0x8000e274        0x0 c:/ti/ccsv5/tools/compiler/gcc-arm-none-eabi-4_7-2012q4/bin/../lib/gcc/arm-none-eabi/4.7.3/../../../../arm-none-eabi/lib\libc.a(lib_a-strcmp.o)
 .bss           0x8000e274        0x0 c:/ti/ccsv5/tools/compiler/gcc-arm-none-eabi-4_7-2012q4/bin/../lib/gcc/arm-none-eabi/4.7.3/../../../../arm-none-eabi/lib\libc.a(lib_a-vfiprintf.o)
 .bss           0x8000e274        0x0 c:/ti/ccsv5/tools/compiler/gcc-arm-none-eabi-4_7-2012q4/bin/../lib/gcc/arm-none-eabi/4.7.3/../../../../arm-none-eabi/lib\libc.a(lib_a-writer.o)
 .bss           0x8000e274        0x0 c:/ti/ccsv5/tools/compiler/gcc-arm-none-eabi-4_7-2012q4/bin/../lib/gcc/arm-none-eabi/4.7.3/../../../../arm-none-eabi/lib\libc.a(lib_a-callocr.o)
 .bss           0x8000e274        0x0 c:/ti/ccsv5/tools/compiler/gcc-arm-none-eabi-4_7-2012q4/bin/../lib/gcc/arm-none-eabi/4.7.3/../../../../arm-none-eabi/lib\libc.a(lib_a-closer.o)
 .bss           0x8000e274        0x0 c:/ti/ccsv5/tools/compiler/gcc-arm-none-eabi-4_7-2012q4/bin/../lib/gcc/arm-none-eabi/4.7.3/../../../../arm-none-eabi/lib\libc.a(lib_a-fclose.o)
 .bss           0x8000e274        0x0 c:/ti/ccsv5/tools/compiler/gcc-arm-none-eabi-4_7-2012q4/bin/../lib/gcc/arm-none-eabi/4.7.3/../../../../arm-none-eabi/lib\libc.a(lib_a-fputwc.o)
 .bss           0x8000e274        0x0 c:/ti/ccsv5/tools/compiler/gcc-arm-none-eabi-4_7-2012q4/bin/../lib/gcc/arm-none-eabi/4.7.3/../../../../arm-none-eabi/lib\libc.a(lib_a-fstatr.o)
 .bss           0x8000e274        0x0 c:/ti/ccsv5/tools/compiler/gcc-arm-none-eabi-4_7-2012q4/bin/../lib/gcc/arm-none-eabi/4.7.3/../../../../arm-none-eabi/lib\libc.a(lib_a-isattyr.o)
 .bss           0x8000e274        0x0 c:/ti/ccsv5/tools/compiler/gcc-arm-none-eabi-4_7-2012q4/bin/../lib/gcc/arm-none-eabi/4.7.3/../../../../arm-none-eabi/lib\libc.a(lib_a-lseekr.o)
 .bss           0x8000e274        0x0 c:/ti/ccsv5/tools/compiler/gcc-arm-none-eabi-4_7-2012q4/bin/../lib/gcc/arm-none-eabi/4.7.3/../../../../arm-none-eabi/lib\libc.a(lib_a-readr.o)
 .bss           0x8000e274        0x0 c:/ti/ccsv5/tools/compiler/gcc-arm-none-eabi-4_7-2012q4/bin/../lib/gcc/arm-none-eabi/4.7.3/../../../../arm-none-eabi/lib\libc.a(lib_a-reent.o)
 .bss           0x8000e274        0x0 c:/ti/ccsv5/tools/compiler/gcc-arm-none-eabi-4_7-2012q4/bin/../lib/gcc/arm-none-eabi/4.7.3/../../../../arm-none-eabi/lib\libc.a(lib_a-wbuf.o)
 .bss           0x8000e274        0x0 c:/ti/ccsv5/tools/compiler/gcc-arm-none-eabi-4_7-2012q4/bin/../lib/gcc/arm-none-eabi/4.7.3/../../../../arm-none-eabi/lib\libc.a(lib_a-wcrtomb.o)
 .bss           0x8000e274        0x0 c:/ti/ccsv5/tools/compiler/gcc-arm-none-eabi-4_7-2012q4/bin/../lib/gcc/arm-none-eabi/4.7.3/../../../../arm-none-eabi/lib\libc.a(lib_a-wctomb_r.o)
 .bss           0x8000e274        0x0 c:/ti/ccsv5/tools/compiler/gcc-arm-none-eabi-4_7-2012q4/bin/../lib/gcc/arm-none-eabi/4.7.3\libgcc.a(_udivsi3.o)
 .bss           0x8000e274        0x0 c:/ti/ccsv5/tools/compiler/gcc-arm-none-eabi-4_7-2012q4/bin/../lib/gcc/arm-none-eabi/4.7.3\libgcc.a(_dvmd_tls.o)
 .bss           0x8000e274        0x0 c:/ti/ccsv5/tools/compiler/gcc-arm-none-eabi-4_7-2012q4/bin/../lib/gcc/arm-none-eabi/4.7.3\libgcc.a(_arm_addsubdf3.o)
 .bss           0x8000e274        0x0 c:/ti/ccsv5/tools/compiler/gcc-arm-none-eabi-4_7-2012q4/bin/../lib/gcc/arm-none-eabi/4.7.3\libgcc.a(_arm_muldivdf3.o)
 .bss           0x8000e274        0x0 c:/ti/ccsv5/tools/compiler/gcc-arm-none-eabi-4_7-2012q4/bin/../lib/gcc/arm-none-eabi/4.7.3\libgcc.a(_arm_cmpdf2.o)
 .bss           0x8000e274        0x0 c:/ti/ccsv5/tools/compiler/gcc-arm-none-eabi-4_7-2012q4/bin/../lib/gcc/arm-none-eabi/4.7.3\libgcc.a(_arm_fixdfsi.o)
 .bss           0x8000e274        0x0 c:/ti/ccsv5/tools/compiler/gcc-arm-none-eabi-4_7-2012q4/bin/../lib/gcc/arm-none-eabi/4.7.3\libgcc.a(_aeabi_uldivmod.o)
 .bss           0x8000e274        0x0 c:/ti/ccsv5/tools/compiler/gcc-arm-none-eabi-4_7-2012q4/bin/../lib/gcc/arm-none-eabi/4.7.3\libgcc.a(bpabi.o)
 .bss           0x8000e274        0x0 c:/ti/ccsv5/tools/compiler/gcc-arm-none-eabi-4_7-2012q4/bin/../lib/gcc/arm-none-eabi/4.7.3\libgcc.a(_divdi3.o)
 .bss           0x8000e274        0x0 c:/ti/ccsv5/tools/compiler/gcc-arm-none-eabi-4_7-2012q4/bin/../lib/gcc/arm-none-eabi/4.7.3\libgcc.a(_udivdi3.o)
 .bss           0x8000e274        0x0 c:/ti/ccsv5/tools/compiler/gcc-arm-none-eabi-4_7-2012q4/bin/../lib/gcc/arm-none-eabi/4.7.3\libgcc.a(_clzsi2.o)
 .bss           0x8000e274        0x0 c:/ti/ccsv5/tools/compiler/gcc-arm-none-eabi-4_7-2012q4/bin/../lib/gcc/arm-none-eabi/4.7.3/../../../../arm-none-eabi/lib\librdimon.a(rdimon-syscalls.o)
 .bss.monitor_stdout
                0x8000e274        0x4 c:/ti/ccsv5/tools/compiler/gcc-arm-none-eabi-4_7-2012q4/bin/../lib/gcc/arm-none-eabi/4.7.3/../../../../arm-none-eabi/lib\librdimon.a(rdimon-syscalls.o)
 .bss.monitor_stdin
                0x8000e278        0x4 c:/ti/ccsv5/tools/compiler/gcc-arm-none-eabi-4_7-2012q4/bin/../lib/gcc/arm-none-eabi/4.7.3/../../../../arm-none-eabi/lib\librdimon.a(rdimon-syscalls.o)
 .bss.monitor_stderr
                0x8000e27c        0x4 c:/ti/ccsv5/tools/compiler/gcc-arm-none-eabi-4_7-2012q4/bin/../lib/gcc/arm-none-eabi/4.7.3/../../../../arm-none-eabi/lib\librdimon.a(rdimon-syscalls.o)
 .bss.heap_end.5738
                0x8000e280        0x4 c:/ti/ccsv5/tools/compiler/gcc-arm-none-eabi-4_7-2012q4/bin/../lib/gcc/arm-none-eabi/4.7.3/../../../../arm-none-eabi/lib\librdimon.a(rdimon-syscalls.o)
 .bss.openfiles
                0x8000e284       0xa0 c:/ti/ccsv5/tools/compiler/gcc-arm-none-eabi-4_7-2012q4/bin/../lib/gcc/arm-none-eabi/4.7.3/../../../../arm-none-eabi/lib\librdimon.a(rdimon-syscalls.o)
 .bss           0x8000e324        0x0 c:/ti/ccsv5/tools/compiler/gcc-arm-none-eabi-4_7-2012q4/bin/../lib/gcc/arm-none-eabi/4.7.3/../../../../arm-none-eabi/lib\librdimon.a(rdimon-_exit.o)
 .bss           0x8000e324        0x0 c:/ti/ccsv5/tools/compiler/gcc-arm-none-eabi-4_7-2012q4/bin/../lib/gcc/arm-none-eabi/4.7.3/../../../../arm-none-eabi/lib\librdimon.a(rdimon-_kill.o)
 .bss           0x8000e324        0x0 c:/ti/ccsv5/tools/compiler/gcc-arm-none-eabi-4_7-2012q4/bin/../lib/gcc/arm-none-eabi/4.7.3/../../../../arm-none-eabi/lib\libc.a(lib_a-errno.o)
 .bss           0x8000e324        0x0 c:/ti/ccsv5/tools/compiler/gcc-arm-none-eabi-4_7-2012q4/bin/../lib/gcc/arm-none-eabi/4.7.3/crtend.o
 .bss           0x8000e324        0x0 c:/ti/ccsv5/tools/compiler/gcc-arm-none-eabi-4_7-2012q4/bin/../lib/gcc/arm-none-eabi/4.7.3/crtn.o
 *(COMMON)
 COMMON         0x8000e324        0x4 c:/ti/ccsv5/tools/compiler/gcc-arm-none-eabi-4_7-2012q4/bin/../lib/gcc/arm-none-eabi/4.7.3/../../../../arm-none-eabi/lib\libc.a(lib_a-reent.o)
                0x8000e324                errno
                0x8000e328                __bss_end__ = .

.heap           0x8000e330     0x4000
                0x8000e330                . = ALIGN (0x4)
                0x8000e330                __end__ = .
                0x8000e330                end = __end__
                0x8000e330                __HeapBase = __end__
 *(.heap*)
 .heap          0x8000e330        0x0 ./startup_ARMCA8.o
                0x80012330                . = (. + HEAPSIZE)
 *fill*         0x8000e330     0x4000 00
                0x80012330                __HeapLimit = .

.stack          0x80012330     0x1000
                0x80012330                . = ALIGN (0x4)
                0x80012330                __StackLimit = .
 *(.stack*)
 .stack         0x80012330        0x0 ./startup_ARMCA8.o
                0x80013330                . = (. + STACKSIZE)
 *fill*         0x80012330     0x1000 00
                0x80013330                __StackTop = .
                0x80013330                __StackBase = .
                0x80013330                PROVIDE (__stack, __StackTop)
START GROUP
LOAD c:/ti/ccsv5/tools/compiler/gcc-arm-none-eabi-4_7-2012q4/bin/../lib/gcc/arm-none-eabi/4.7.3\libgcc.a
LOAD c:/ti/ccsv5/tools/compiler/gcc-arm-none-eabi-4_7-2012q4/bin/../lib/gcc/arm-none-eabi/4.7.3/../../../../arm-none-eabi/lib\libg.a
LOAD c:/ti/ccsv5/tools/compiler/gcc-arm-none-eabi-4_7-2012q4/bin/../lib/gcc/arm-none-eabi/4.7.3/../../../../arm-none-eabi/lib\libc.a
END GROUP
LOAD c:/ti/ccsv5/tools/compiler/gcc-arm-none-eabi-4_7-2012q4/bin/../lib/gcc/arm-none-eabi/4.7.3/crtend.o
LOAD c:/ti/ccsv5/tools/compiler/gcc-arm-none-eabi-4_7-2012q4/bin/../lib/gcc/arm-none-eabi/4.7.3/crtn.o
OUTPUT(ARM_DSP_Communication_ARM.out elf32-littlearm)

.ARM.attributes
                0x00000000       0x31
 .ARM.attributes
                0x00000000       0x16 c:/ti/ccsv5/tools/compiler/gcc-arm-none-eabi-4_7-2012q4/bin/../lib/gcc/arm-none-eabi/4.7.3/crti.o
 .ARM.attributes
                0x00000016       0x30 c:/ti/ccsv5/tools/compiler/gcc-arm-none-eabi-4_7-2012q4/bin/../lib/gcc/arm-none-eabi/4.7.3/crtbegin.o
 .ARM.attributes
                0x00000046       0x14 c:/ti/ccsv5/tools/compiler/gcc-arm-none-eabi-4_7-2012q4/bin/../lib/gcc/arm-none-eabi/4.7.3/../../../../arm-none-eabi/lib/rdimon-crt0.o
 .ARM.attributes
                0x0000005a       0x23 ./common_arm/v7_pmu.o
 .ARM.attributes
                0x0000007d       0x23 ./common_arm/utilFxns.o
 .ARM.attributes
                0x000000a0       0x2f ./common_arm/arm_utility.o
 .ARM.attributes
                0x000000cf       0x2f ./common_arm/arm_cpintc.o
 .ARM.attributes
                0x000000fe       0x2f ./common_arm/aintc_inth.o
 .ARM.attributes
                0x0000012d       0x2f ./common_arm/GIC_ctl.o
 .ARM.attributes
                0x0000015c       0x23 ./common_arm/Cortex_A_generic_timer.o
 .ARM.attributes
                0x0000017f       0x23 ./startup_ARMCA8.o
 .ARM.attributes
                0x000001a2       0x2f ./main.o
 .ARM.attributes
                0x000001d1       0x30 c:/ti/ccsv5/tools/compiler/gcc-arm-none-eabi-4_7-2012q4/bin/../lib/gcc/arm-none-eabi/4.7.3/../../../../arm-none-eabi/lib\libc.a(lib_a-__atexit.o)
 .ARM.attributes
                0x00000201       0x30 c:/ti/ccsv5/tools/compiler/gcc-arm-none-eabi-4_7-2012q4/bin/../lib/gcc/arm-none-eabi/4.7.3/../../../../arm-none-eabi/lib\libc.a(lib_a-exit.o)
 .ARM.attributes
                0x00000231       0x30 c:/ti/ccsv5/tools/compiler/gcc-arm-none-eabi-4_7-2012q4/bin/../lib/gcc/arm-none-eabi/4.7.3/../../../../arm-none-eabi/lib\libc.a(lib_a-fini.o)
 .ARM.attributes
                0x00000261       0x30 c:/ti/ccsv5/tools/compiler/gcc-arm-none-eabi-4_7-2012q4/bin/../lib/gcc/arm-none-eabi/4.7.3/../../../../arm-none-eabi/lib\libc.a(lib_a-impure.o)
 .ARM.attributes
                0x00000291       0x30 c:/ti/ccsv5/tools/compiler/gcc-arm-none-eabi-4_7-2012q4/bin/../lib/gcc/arm-none-eabi/4.7.3/../../../../arm-none-eabi/lib\libc.a(lib_a-init.o)
 .ARM.attributes
                0x000002c1       0x30 c:/ti/ccsv5/tools/compiler/gcc-arm-none-eabi-4_7-2012q4/bin/../lib/gcc/arm-none-eabi/4.7.3/../../../../arm-none-eabi/lib\libc.a(lib_a-memset.o)
 .ARM.attributes
                0x000002f1       0x30 c:/ti/ccsv5/tools/compiler/gcc-arm-none-eabi-4_7-2012q4/bin/../lib/gcc/arm-none-eabi/4.7.3/../../../../arm-none-eabi/lib\libc.a(lib_a-printf.o)
 .ARM.attributes
                0x00000321       0x30 c:/ti/ccsv5/tools/compiler/gcc-arm-none-eabi-4_7-2012q4/bin/../lib/gcc/arm-none-eabi/4.7.3/../../../../arm-none-eabi/lib\libc.a(lib_a-puts.o)
 .ARM.attributes
                0x00000351       0x30 c:/ti/ccsv5/tools/compiler/gcc-arm-none-eabi-4_7-2012q4/bin/../lib/gcc/arm-none-eabi/4.7.3/../../../../arm-none-eabi/lib\libc.a(lib_a-strlen.o)
 .ARM.attributes
                0x00000381       0x30 c:/ti/ccsv5/tools/compiler/gcc-arm-none-eabi-4_7-2012q4/bin/../lib/gcc/arm-none-eabi/4.7.3/../../../../arm-none-eabi/lib\libc.a(lib_a-vfprintf.o)
 .ARM.attributes
                0x000003b1       0x30 c:/ti/ccsv5/tools/compiler/gcc-arm-none-eabi-4_7-2012q4/bin/../lib/gcc/arm-none-eabi/4.7.3/../../../../arm-none-eabi/lib\libc.a(lib_a-wsetup.o)
 .ARM.attributes
                0x000003e1       0x30 c:/ti/ccsv5/tools/compiler/gcc-arm-none-eabi-4_7-2012q4/bin/../lib/gcc/arm-none-eabi/4.7.3/../../../../arm-none-eabi/lib\libc.a(lib_a-__call_atexit.o)
 .ARM.attributes
                0x00000411       0x30 c:/ti/ccsv5/tools/compiler/gcc-arm-none-eabi-4_7-2012q4/bin/../lib/gcc/arm-none-eabi/4.7.3/../../../../arm-none-eabi/lib\libc.a(lib_a-atexit.o)
 .ARM.attributes
                0x00000441       0x30 c:/ti/ccsv5/tools/compiler/gcc-arm-none-eabi-4_7-2012q4/bin/../lib/gcc/arm-none-eabi/4.7.3/../../../../arm-none-eabi/lib\libc.a(lib_a-dtoa.o)
 .ARM.attributes
                0x00000471       0x30 c:/ti/ccsv5/tools/compiler/gcc-arm-none-eabi-4_7-2012q4/bin/../lib/gcc/arm-none-eabi/4.7.3/../../../../arm-none-eabi/lib\libc.a(lib_a-fflush.o)
 .ARM.attributes
                0x000004a1       0x30 c:/ti/ccsv5/tools/compiler/gcc-arm-none-eabi-4_7-2012q4/bin/../lib/gcc/arm-none-eabi/4.7.3/../../../../arm-none-eabi/lib\libc.a(lib_a-findfp.o)
 .ARM.attributes
                0x000004d1       0x30 c:/ti/ccsv5/tools/compiler/gcc-arm-none-eabi-4_7-2012q4/bin/../lib/gcc/arm-none-eabi/4.7.3/../../../../arm-none-eabi/lib\libc.a(lib_a-freer.o)
 .ARM.attributes
                0x00000501       0x30 c:/ti/ccsv5/tools/compiler/gcc-arm-none-eabi-4_7-2012q4/bin/../lib/gcc/arm-none-eabi/4.7.3/../../../../arm-none-eabi/lib\libc.a(lib_a-fvwrite.o)
 .ARM.attributes
                0x00000531       0x30 c:/ti/ccsv5/tools/compiler/gcc-arm-none-eabi-4_7-2012q4/bin/../lib/gcc/arm-none-eabi/4.7.3/../../../../arm-none-eabi/lib\libc.a(lib_a-fwalk.o)
 .ARM.attributes
                0x00000561       0x30 c:/ti/ccsv5/tools/compiler/gcc-arm-none-eabi-4_7-2012q4/bin/../lib/gcc/arm-none-eabi/4.7.3/../../../../arm-none-eabi/lib\libc.a(lib_a-locale.o)
 .ARM.attributes
                0x00000591       0x30 c:/ti/ccsv5/tools/compiler/gcc-arm-none-eabi-4_7-2012q4/bin/../lib/gcc/arm-none-eabi/4.7.3/../../../../arm-none-eabi/lib\libc.a(lib_a-makebuf.o)
 .ARM.attributes
                0x000005c1       0x30 c:/ti/ccsv5/tools/compiler/gcc-arm-none-eabi-4_7-2012q4/bin/../lib/gcc/arm-none-eabi/4.7.3/../../../../arm-none-eabi/lib\libc.a(lib_a-mallocr.o)
 .ARM.attributes
                0x000005f1       0x30 c:/ti/ccsv5/tools/compiler/gcc-arm-none-eabi-4_7-2012q4/bin/../lib/gcc/arm-none-eabi/4.7.3/../../../../arm-none-eabi/lib\libc.a(lib_a-memchr.o)
 .ARM.attributes
                0x00000621       0x30 c:/ti/ccsv5/tools/compiler/gcc-arm-none-eabi-4_7-2012q4/bin/../lib/gcc/arm-none-eabi/4.7.3/../../../../arm-none-eabi/lib\libc.a(lib_a-memcpy.o)
 .ARM.attributes
                0x00000651       0x30 c:/ti/ccsv5/tools/compiler/gcc-arm-none-eabi-4_7-2012q4/bin/../lib/gcc/arm-none-eabi/4.7.3/../../../../arm-none-eabi/lib\libc.a(lib_a-memmove.o)
 .ARM.attributes
                0x00000681       0x30 c:/ti/ccsv5/tools/compiler/gcc-arm-none-eabi-4_7-2012q4/bin/../lib/gcc/arm-none-eabi/4.7.3/../../../../arm-none-eabi/lib\libc.a(lib_a-mlock.o)
 .ARM.attributes
                0x000006b1       0x30 c:/ti/ccsv5/tools/compiler/gcc-arm-none-eabi-4_7-2012q4/bin/../lib/gcc/arm-none-eabi/4.7.3/../../../../arm-none-eabi/lib\libc.a(lib_a-mprec.o)
 .ARM.attributes
                0x000006e1       0x30 c:/ti/ccsv5/tools/compiler/gcc-arm-none-eabi-4_7-2012q4/bin/../lib/gcc/arm-none-eabi/4.7.3/../../../../arm-none-eabi/lib\libc.a(lib_a-reallocr.o)
 .ARM.attributes
                0x00000711       0x30 c:/ti/ccsv5/tools/compiler/gcc-arm-none-eabi-4_7-2012q4/bin/../lib/gcc/arm-none-eabi/4.7.3/../../../../arm-none-eabi/lib\libc.a(lib_a-s_fpclassify.o)
 .ARM.attributes
                0x00000741       0x30 c:/ti/ccsv5/tools/compiler/gcc-arm-none-eabi-4_7-2012q4/bin/../lib/gcc/arm-none-eabi/4.7.3/../../../../arm-none-eabi/lib\libc.a(lib_a-sbrkr.o)
 .ARM.attributes
                0x00000771       0x30 c:/ti/ccsv5/tools/compiler/gcc-arm-none-eabi-4_7-2012q4/bin/../lib/gcc/arm-none-eabi/4.7.3/../../../../arm-none-eabi/lib\libc.a(lib_a-stdio.o)
 .ARM.attributes
                0x000007a1       0x30 c:/ti/ccsv5/tools/compiler/gcc-arm-none-eabi-4_7-2012q4/bin/../lib/gcc/arm-none-eabi/4.7.3/../../../../arm-none-eabi/lib\libc.a(lib_a-strcmp.o)
 .ARM.attributes
                0x000007d1       0x30 c:/ti/ccsv5/tools/compiler/gcc-arm-none-eabi-4_7-2012q4/bin/../lib/gcc/arm-none-eabi/4.7.3/../../../../arm-none-eabi/lib\libc.a(lib_a-vfiprintf.o)
 .ARM.attributes
                0x00000801       0x30 c:/ti/ccsv5/tools/compiler/gcc-arm-none-eabi-4_7-2012q4/bin/../lib/gcc/arm-none-eabi/4.7.3/../../../../arm-none-eabi/lib\libc.a(lib_a-writer.o)
 .ARM.attributes
                0x00000831       0x30 c:/ti/ccsv5/tools/compiler/gcc-arm-none-eabi-4_7-2012q4/bin/../lib/gcc/arm-none-eabi/4.7.3/../../../../arm-none-eabi/lib\libc.a(lib_a-callocr.o)
 .ARM.attributes
                0x00000861       0x30 c:/ti/ccsv5/tools/compiler/gcc-arm-none-eabi-4_7-2012q4/bin/../lib/gcc/arm-none-eabi/4.7.3/../../../../arm-none-eabi/lib\libc.a(lib_a-closer.o)
 .ARM.attributes
                0x00000891       0x30 c:/ti/ccsv5/tools/compiler/gcc-arm-none-eabi-4_7-2012q4/bin/../lib/gcc/arm-none-eabi/4.7.3/../../../../arm-none-eabi/lib\libc.a(lib_a-fclose.o)
 .ARM.attributes
                0x000008c1       0x30 c:/ti/ccsv5/tools/compiler/gcc-arm-none-eabi-4_7-2012q4/bin/../lib/gcc/arm-none-eabi/4.7.3/../../../../arm-none-eabi/lib\libc.a(lib_a-fputwc.o)
 .ARM.attributes
                0x000008f1       0x30 c:/ti/ccsv5/tools/compiler/gcc-arm-none-eabi-4_7-2012q4/bin/../lib/gcc/arm-none-eabi/4.7.3/../../../../arm-none-eabi/lib\libc.a(lib_a-fstatr.o)
 .ARM.attributes
                0x00000921       0x30 c:/ti/ccsv5/tools/compiler/gcc-arm-none-eabi-4_7-2012q4/bin/../lib/gcc/arm-none-eabi/4.7.3/../../../../arm-none-eabi/lib\libc.a(lib_a-isattyr.o)
 .ARM.attributes
                0x00000951       0x30 c:/ti/ccsv5/tools/compiler/gcc-arm-none-eabi-4_7-2012q4/bin/../lib/gcc/arm-none-eabi/4.7.3/../../../../arm-none-eabi/lib\libc.a(lib_a-lseekr.o)
 .ARM.attributes
                0x00000981       0x30 c:/ti/ccsv5/tools/compiler/gcc-arm-none-eabi-4_7-2012q4/bin/../lib/gcc/arm-none-eabi/4.7.3/../../../../arm-none-eabi/lib\libc.a(lib_a-readr.o)
 .ARM.attributes
                0x000009b1       0x30 c:/ti/ccsv5/tools/compiler/gcc-arm-none-eabi-4_7-2012q4/bin/../lib/gcc/arm-none-eabi/4.7.3/../../../../arm-none-eabi/lib\libc.a(lib_a-reent.o)
 .ARM.attributes
                0x000009e1       0x30 c:/ti/ccsv5/tools/compiler/gcc-arm-none-eabi-4_7-2012q4/bin/../lib/gcc/arm-none-eabi/4.7.3/../../../../arm-none-eabi/lib\libc.a(lib_a-wbuf.o)
 .ARM.attributes
                0x00000a11       0x30 c:/ti/ccsv5/tools/compiler/gcc-arm-none-eabi-4_7-2012q4/bin/../lib/gcc/arm-none-eabi/4.7.3/../../../../arm-none-eabi/lib\libc.a(lib_a-wcrtomb.o)
 .ARM.attributes
                0x00000a41       0x30 c:/ti/ccsv5/tools/compiler/gcc-arm-none-eabi-4_7-2012q4/bin/../lib/gcc/arm-none-eabi/4.7.3/../../../../arm-none-eabi/lib\libc.a(lib_a-wctomb_r.o)
 .ARM.attributes
                0x00000a71       0x18 c:/ti/ccsv5/tools/compiler/gcc-arm-none-eabi-4_7-2012q4/bin/../lib/gcc/arm-none-eabi/4.7.3\libgcc.a(_udivsi3.o)
 .ARM.attributes
                0x00000a89       0x18 c:/ti/ccsv5/tools/compiler/gcc-arm-none-eabi-4_7-2012q4/bin/../lib/gcc/arm-none-eabi/4.7.3\libgcc.a(_dvmd_tls.o)
 .ARM.attributes
                0x00000aa1       0x18 c:/ti/ccsv5/tools/compiler/gcc-arm-none-eabi-4_7-2012q4/bin/../lib/gcc/arm-none-eabi/4.7.3\libgcc.a(_arm_addsubdf3.o)
 .ARM.attributes
                0x00000ab9       0x18 c:/ti/ccsv5/tools/compiler/gcc-arm-none-eabi-4_7-2012q4/bin/../lib/gcc/arm-none-eabi/4.7.3\libgcc.a(_arm_muldivdf3.o)
 .ARM.attributes
                0x00000ad1       0x18 c:/ti/ccsv5/tools/compiler/gcc-arm-none-eabi-4_7-2012q4/bin/../lib/gcc/arm-none-eabi/4.7.3\libgcc.a(_arm_cmpdf2.o)
 .ARM.attributes
                0x00000ae9       0x18 c:/ti/ccsv5/tools/compiler/gcc-arm-none-eabi-4_7-2012q4/bin/../lib/gcc/arm-none-eabi/4.7.3\libgcc.a(_arm_fixdfsi.o)
 .ARM.attributes
                0x00000b01       0x18 c:/ti/ccsv5/tools/compiler/gcc-arm-none-eabi-4_7-2012q4/bin/../lib/gcc/arm-none-eabi/4.7.3\libgcc.a(_aeabi_uldivmod.o)
 .ARM.attributes
                0x00000b19       0x30 c:/ti/ccsv5/tools/compiler/gcc-arm-none-eabi-4_7-2012q4/bin/../lib/gcc/arm-none-eabi/4.7.3\libgcc.a(bpabi.o)
 .ARM.attributes
                0x00000b49       0x30 c:/ti/ccsv5/tools/compiler/gcc-arm-none-eabi-4_7-2012q4/bin/../lib/gcc/arm-none-eabi/4.7.3\libgcc.a(_divdi3.o)
 .ARM.attributes
                0x00000b79       0x30 c:/ti/ccsv5/tools/compiler/gcc-arm-none-eabi-4_7-2012q4/bin/../lib/gcc/arm-none-eabi/4.7.3\libgcc.a(_udivdi3.o)
 .ARM.attributes
                0x00000ba9       0x18 c:/ti/ccsv5/tools/compiler/gcc-arm-none-eabi-4_7-2012q4/bin/../lib/gcc/arm-none-eabi/4.7.3\libgcc.a(_clzsi2.o)
 .ARM.attributes
                0x00000bc1       0x30 c:/ti/ccsv5/tools/compiler/gcc-arm-none-eabi-4_7-2012q4/bin/../lib/gcc/arm-none-eabi/4.7.3/../../../../arm-none-eabi/lib\librdimon.a(rdimon-syscalls.o)
 .ARM.attributes
                0x00000bf1       0x30 c:/ti/ccsv5/tools/compiler/gcc-arm-none-eabi-4_7-2012q4/bin/../lib/gcc/arm-none-eabi/4.7.3/../../../../arm-none-eabi/lib\librdimon.a(rdimon-_exit.o)
 .ARM.attributes
                0x00000c21       0x30 c:/ti/ccsv5/tools/compiler/gcc-arm-none-eabi-4_7-2012q4/bin/../lib/gcc/arm-none-eabi/4.7.3/../../../../arm-none-eabi/lib\librdimon.a(rdimon-_kill.o)
 .ARM.attributes
                0x00000c51       0x30 c:/ti/ccsv5/tools/compiler/gcc-arm-none-eabi-4_7-2012q4/bin/../lib/gcc/arm-none-eabi/4.7.3/../../../../arm-none-eabi/lib\libc.a(lib_a-errno.o)
 .ARM.attributes
                0x00000c81       0x30 c:/ti/ccsv5/tools/compiler/gcc-arm-none-eabi-4_7-2012q4/bin/../lib/gcc/arm-none-eabi/4.7.3/crtend.o
 .ARM.attributes
                0x00000cb1       0x18 c:/ti/ccsv5/tools/compiler/gcc-arm-none-eabi-4_7-2012q4/bin/../lib/gcc/arm-none-eabi/4.7.3/crtn.o

.comment        0x00000000       0x70
 .comment       0x00000000       0x70 ./common_arm/arm_utility.o
                                 0x71 (size before relaxing)
 .comment       0x00000000       0x71 ./common_arm/arm_cpintc.o
 .comment       0x00000000       0x71 ./common_arm/aintc_inth.o
 .comment       0x00000000       0x71 ./common_arm/GIC_ctl.o
 .comment       0x00000000       0x71 ./main.o

.debug_line     0x00000000      0x9a2
 .debug_line    0x00000000       0xb2 ./common_arm/v7_pmu.o
 .debug_line    0x000000b2       0x49 ./common_arm/utilFxns.o
 .debug_line    0x000000fb      0x30b ./common_arm/arm_utility.o
 .debug_line    0x00000406       0xc4 ./common_arm/arm_cpintc.o
 .debug_line    0x000004ca      0x147 ./common_arm/aintc_inth.o
 .debug_line    0x00000611      0x1aa ./common_arm/GIC_ctl.o
 .debug_line    0x000007bb       0x79 ./common_arm/Cortex_A_generic_timer.o
 .debug_line    0x00000834       0x79 ./startup_ARMCA8.o
 .debug_line    0x000008ad       0xf5 ./main.o

.debug_info     0x00000000     0x3694
 .debug_info    0x00000000       0x71 ./common_arm/v7_pmu.o
 .debug_info    0x00000071       0x73 ./common_arm/utilFxns.o
 .debug_info    0x000000e4      0x44e ./common_arm/arm_utility.o
 .debug_info    0x00000532      0x5f5 ./common_arm/arm_cpintc.o
 .debug_info    0x00000b27      0xe70 ./common_arm/aintc_inth.o
 .debug_info    0x00001997     0x1209 ./common_arm/GIC_ctl.o
 .debug_info    0x00002ba0       0x81 ./common_arm/Cortex_A_generic_timer.o
 .debug_info    0x00002c21       0x6a ./startup_ARMCA8.o
 .debug_info    0x00002c8b      0xa09 ./main.o

.debug_abbrev   0x00000000      0x8e2
 .debug_abbrev  0x00000000       0x14 ./common_arm/v7_pmu.o
 .debug_abbrev  0x00000014       0x14 ./common_arm/utilFxns.o
 .debug_abbrev  0x00000028      0x1b5 ./common_arm/arm_utility.o
 .debug_abbrev  0x000001dd      0x116 ./common_arm/arm_cpintc.o
 .debug_abbrev  0x000002f3      0x1d4 ./common_arm/aintc_inth.o
 .debug_abbrev  0x000004c7      0x299 ./common_arm/GIC_ctl.o
 .debug_abbrev  0x00000760       0x14 ./common_arm/Cortex_A_generic_timer.o
 .debug_abbrev  0x00000774       0x12 ./startup_ARMCA8.o
 .debug_abbrev  0x00000786      0x15c ./main.o

.debug_aranges  0x00000000      0x130
 .debug_aranges
                0x00000000       0x20 ./common_arm/v7_pmu.o
 .debug_aranges
                0x00000020       0x20 ./common_arm/utilFxns.o
 .debug_aranges
                0x00000040       0x20 ./common_arm/arm_utility.o
 .debug_aranges
                0x00000060       0x20 ./common_arm/arm_cpintc.o
 .debug_aranges
                0x00000080       0x20 ./common_arm/aintc_inth.o
 .debug_aranges
                0x000000a0       0x20 ./common_arm/GIC_ctl.o
 .debug_aranges
                0x000000c0       0x20 ./common_arm/Cortex_A_generic_timer.o
 .debug_aranges
                0x000000e0       0x28 ./startup_ARMCA8.o
 .debug_aranges
                0x00000108       0x28 ./main.o

.debug_loc      0x00000000      0xeb1
 .debug_loc     0x00000000      0x67d ./common_arm/arm_utility.o
 .debug_loc     0x0000067d       0x5f ./common_arm/arm_cpintc.o
 .debug_loc     0x000006dc      0x33e ./common_arm/aintc_inth.o
 .debug_loc     0x00000a1a      0x444 ./common_arm/GIC_ctl.o
 .debug_loc     0x00000e5e       0x53 ./main.o

.debug_str      0x00000000     0x1214
 .debug_str     0x00000000      0x2cd ./common_arm/arm_utility.o
                                0x30e (size before relaxing)
 .debug_str     0x000002cd      0x591 ./common_arm/arm_cpintc.o
                                0x6d3 (size before relaxing)
 .debug_str     0x0000085e      0x7a3 ./common_arm/aintc_inth.o
                                0x8bf (size before relaxing)
 .debug_str     0x00001001      0x1e0 ./common_arm/GIC_ctl.o
                                0x8c3 (size before relaxing)
 .debug_str     0x000011e1       0x33 ./main.o
                                0x53d (size before relaxing)

.debug_frame    0x00000000     0x1664
 .debug_frame   0x00000000      0x114 ./common_arm/arm_utility.o
 .debug_frame   0x00000114       0x60 ./common_arm/arm_cpintc.o
 .debug_frame   0x00000174      0x150 ./common_arm/aintc_inth.o
 .debug_frame   0x000002c4      0x130 ./common_arm/GIC_ctl.o
 .debug_frame   0x000003f4       0x50 ./main.o
 .debug_frame   0x00000444       0x34 c:/ti/ccsv5/tools/compiler/gcc-arm-none-eabi-4_7-2012q4/bin/../lib/gcc/arm-none-eabi/4.7.3/../../../../arm-none-eabi/lib\libc.a(lib_a-__atexit.o)
 .debug_frame   0x00000478       0x28 c:/ti/ccsv5/tools/compiler/gcc-arm-none-eabi-4_7-2012q4/bin/../lib/gcc/arm-none-eabi/4.7.3/../../../../arm-none-eabi/lib\libc.a(lib_a-exit.o)
 .debug_frame   0x000004a0       0x2c c:/ti/ccsv5/tools/compiler/gcc-arm-none-eabi-4_7-2012q4/bin/../lib/gcc/arm-none-eabi/4.7.3/../../../../arm-none-eabi/lib\libc.a(lib_a-fini.o)
 .debug_frame   0x000004cc       0x2c c:/ti/ccsv5/tools/compiler/gcc-arm-none-eabi-4_7-2012q4/bin/../lib/gcc/arm-none-eabi/4.7.3/../../../../arm-none-eabi/lib\libc.a(lib_a-init.o)
 .debug_frame   0x000004f8       0x28 c:/ti/ccsv5/tools/compiler/gcc-arm-none-eabi-4_7-2012q4/bin/../lib/gcc/arm-none-eabi/4.7.3/../../../../arm-none-eabi/lib\libc.a(lib_a-memset.o)
 .debug_frame   0x00000520       0x58 c:/ti/ccsv5/tools/compiler/gcc-arm-none-eabi-4_7-2012q4/bin/../lib/gcc/arm-none-eabi/4.7.3/../../../../arm-none-eabi/lib\libc.a(lib_a-printf.o)
 .debug_frame   0x00000578       0x3c c:/ti/ccsv5/tools/compiler/gcc-arm-none-eabi-4_7-2012q4/bin/../lib/gcc/arm-none-eabi/4.7.3/../../../../arm-none-eabi/lib\libc.a(lib_a-puts.o)
 .debug_frame   0x000005b4       0x20 c:/ti/ccsv5/tools/compiler/gcc-arm-none-eabi-4_7-2012q4/bin/../lib/gcc/arm-none-eabi/4.7.3/../../../../arm-none-eabi/lib\libc.a(lib_a-strlen.o)
 .debug_frame   0x000005d4       0x58 c:/ti/ccsv5/tools/compiler/gcc-arm-none-eabi-4_7-2012q4/bin/../lib/gcc/arm-none-eabi/4.7.3/../../../../arm-none-eabi/lib\libc.a(lib_a-vfprintf.o)
 .debug_frame   0x0000062c       0x2c c:/ti/ccsv5/tools/compiler/gcc-arm-none-eabi-4_7-2012q4/bin/../lib/gcc/arm-none-eabi/4.7.3/../../../../arm-none-eabi/lib\libc.a(lib_a-wsetup.o)
 .debug_frame   0x00000658       0x50 c:/ti/ccsv5/tools/compiler/gcc-arm-none-eabi-4_7-2012q4/bin/../lib/gcc/arm-none-eabi/4.7.3/../../../../arm-none-eabi/lib\libc.a(lib_a-__call_atexit.o)
 .debug_frame   0x000006a8       0x28 c:/ti/ccsv5/tools/compiler/gcc-arm-none-eabi-4_7-2012q4/bin/../lib/gcc/arm-none-eabi/4.7.3/../../../../arm-none-eabi/lib\libc.a(lib_a-atexit.o)
 .debug_frame   0x000006d0       0x64 c:/ti/ccsv5/tools/compiler/gcc-arm-none-eabi-4_7-2012q4/bin/../lib/gcc/arm-none-eabi/4.7.3/../../../../arm-none-eabi/lib\libc.a(lib_a-dtoa.o)
 .debug_frame   0x00000734       0x48 c:/ti/ccsv5/tools/compiler/gcc-arm-none-eabi-4_7-2012q4/bin/../lib/gcc/arm-none-eabi/4.7.3/../../../../arm-none-eabi/lib\libc.a(lib_a-fflush.o)
 .debug_frame   0x0000077c      0x134 c:/ti/ccsv5/tools/compiler/gcc-arm-none-eabi-4_7-2012q4/bin/../lib/gcc/arm-none-eabi/4.7.3/../../../../arm-none-eabi/lib\libc.a(lib_a-findfp.o)
 .debug_frame   0x000008b0       0x50 c:/ti/ccsv5/tools/compiler/gcc-arm-none-eabi-4_7-2012q4/bin/../lib/gcc/arm-none-eabi/4.7.3/../../../../arm-none-eabi/lib\libc.a(lib_a-freer.o)
 .debug_frame   0x00000900       0x38 c:/ti/ccsv5/tools/compiler/gcc-arm-none-eabi-4_7-2012q4/bin/../lib/gcc/arm-none-eabi/4.7.3/../../../../arm-none-eabi/lib\libc.a(lib_a-fvwrite.o)
 .debug_frame   0x00000938       0x54 c:/ti/ccsv5/tools/compiler/gcc-arm-none-eabi-4_7-2012q4/bin/../lib/gcc/arm-none-eabi/4.7.3/../../../../arm-none-eabi/lib\libc.a(lib_a-fwalk.o)
 .debug_frame   0x0000098c       0x98 c:/ti/ccsv5/tools/compiler/gcc-arm-none-eabi-4_7-2012q4/bin/../lib/gcc/arm-none-eabi/4.7.3/../../../../arm-none-eabi/lib\libc.a(lib_a-locale.o)
 .debug_frame   0x00000a24       0x30 c:/ti/ccsv5/tools/compiler/gcc-arm-none-eabi-4_7-2012q4/bin/../lib/gcc/arm-none-eabi/4.7.3/../../../../arm-none-eabi/lib\libc.a(lib_a-makebuf.o)
 .debug_frame   0x00000a54       0x38 c:/ti/ccsv5/tools/compiler/gcc-arm-none-eabi-4_7-2012q4/bin/../lib/gcc/arm-none-eabi/4.7.3/../../../../arm-none-eabi/lib\libc.a(lib_a-mallocr.o)
 .debug_frame   0x00000a8c       0x2c c:/ti/ccsv5/tools/compiler/gcc-arm-none-eabi-4_7-2012q4/bin/../lib/gcc/arm-none-eabi/4.7.3/../../../../arm-none-eabi/lib\libc.a(lib_a-memchr.o)
 .debug_frame   0x00000ab8       0x2c c:/ti/ccsv5/tools/compiler/gcc-arm-none-eabi-4_7-2012q4/bin/../lib/gcc/arm-none-eabi/4.7.3/../../../../arm-none-eabi/lib\libc.a(lib_a-memcpy.o)
 .debug_frame   0x00000ae4       0x2c c:/ti/ccsv5/tools/compiler/gcc-arm-none-eabi-4_7-2012q4/bin/../lib/gcc/arm-none-eabi/4.7.3/../../../../arm-none-eabi/lib\libc.a(lib_a-memmove.o)
 .debug_frame   0x00000b10       0x30 c:/ti/ccsv5/tools/compiler/gcc-arm-none-eabi-4_7-2012q4/bin/../lib/gcc/arm-none-eabi/4.7.3/../../../../arm-none-eabi/lib\libc.a(lib_a-mlock.o)
 .debug_frame   0x00000b40      0x220 c:/ti/ccsv5/tools/compiler/gcc-arm-none-eabi-4_7-2012q4/bin/../lib/gcc/arm-none-eabi/4.7.3/../../../../arm-none-eabi/lib\libc.a(lib_a-mprec.o)
 .debug_frame   0x00000d60       0x38 c:/ti/ccsv5/tools/compiler/gcc-arm-none-eabi-4_7-2012q4/bin/../lib/gcc/arm-none-eabi/4.7.3/../../../../arm-none-eabi/lib\libc.a(lib_a-reallocr.o)
 .debug_frame   0x00000d98       0x20 c:/ti/ccsv5/tools/compiler/gcc-arm-none-eabi-4_7-2012q4/bin/../lib/gcc/arm-none-eabi/4.7.3/../../../../arm-none-eabi/lib\libc.a(lib_a-s_fpclassify.o)
 .debug_frame   0x00000db8       0x2c c:/ti/ccsv5/tools/compiler/gcc-arm-none-eabi-4_7-2012q4/bin/../lib/gcc/arm-none-eabi/4.7.3/../../../../arm-none-eabi/lib\libc.a(lib_a-sbrkr.o)
 .debug_frame   0x00000de4       0x88 c:/ti/ccsv5/tools/compiler/gcc-arm-none-eabi-4_7-2012q4/bin/../lib/gcc/arm-none-eabi/4.7.3/../../../../arm-none-eabi/lib\libc.a(lib_a-stdio.o)
 .debug_frame   0x00000e6c       0x30 c:/ti/ccsv5/tools/compiler/gcc-arm-none-eabi-4_7-2012q4/bin/../lib/gcc/arm-none-eabi/4.7.3/../../../../arm-none-eabi/lib\libc.a(lib_a-strcmp.o)
 .debug_frame   0x00000e9c       0x7c c:/ti/ccsv5/tools/compiler/gcc-arm-none-eabi-4_7-2012q4/bin/../lib/gcc/arm-none-eabi/4.7.3/../../../../arm-none-eabi/lib\libc.a(lib_a-vfiprintf.o)
 .debug_frame   0x00000f18       0x2c c:/ti/ccsv5/tools/compiler/gcc-arm-none-eabi-4_7-2012q4/bin/../lib/gcc/arm-none-eabi/4.7.3/../../../../arm-none-eabi/lib\libc.a(lib_a-writer.o)
 .debug_frame   0x00000f44       0x28 c:/ti/ccsv5/tools/compiler/gcc-arm-none-eabi-4_7-2012q4/bin/../lib/gcc/arm-none-eabi/4.7.3/../../../../arm-none-eabi/lib\libc.a(lib_a-callocr.o)
 .debug_frame   0x00000f6c       0x2c c:/ti/ccsv5/tools/compiler/gcc-arm-none-eabi-4_7-2012q4/bin/../lib/gcc/arm-none-eabi/4.7.3/../../../../arm-none-eabi/lib\libc.a(lib_a-closer.o)
 .debug_frame   0x00000f98       0x3c c:/ti/ccsv5/tools/compiler/gcc-arm-none-eabi-4_7-2012q4/bin/../lib/gcc/arm-none-eabi/4.7.3/../../../../arm-none-eabi/lib\libc.a(lib_a-fclose.o)
 .debug_frame   0x00000fd4       0x50 c:/ti/ccsv5/tools/compiler/gcc-arm-none-eabi-4_7-2012q4/bin/../lib/gcc/arm-none-eabi/4.7.3/../../../../arm-none-eabi/lib\libc.a(lib_a-fputwc.o)
 .debug_frame   0x00001024       0x2c c:/ti/ccsv5/tools/compiler/gcc-arm-none-eabi-4_7-2012q4/bin/../lib/gcc/arm-none-eabi/4.7.3/../../../../arm-none-eabi/lib\libc.a(lib_a-fstatr.o)
 .debug_frame   0x00001050       0x2c c:/ti/ccsv5/tools/compiler/gcc-arm-none-eabi-4_7-2012q4/bin/../lib/gcc/arm-none-eabi/4.7.3/../../../../arm-none-eabi/lib\libc.a(lib_a-isattyr.o)
 .debug_frame   0x0000107c       0x2c c:/ti/ccsv5/tools/compiler/gcc-arm-none-eabi-4_7-2012q4/bin/../lib/gcc/arm-none-eabi/4.7.3/../../../../arm-none-eabi/lib\libc.a(lib_a-lseekr.o)
 .debug_frame   0x000010a8       0x2c c:/ti/ccsv5/tools/compiler/gcc-arm-none-eabi-4_7-2012q4/bin/../lib/gcc/arm-none-eabi/4.7.3/../../../../arm-none-eabi/lib\libc.a(lib_a-readr.o)
 .debug_frame   0x000010d4       0x68 c:/ti/ccsv5/tools/compiler/gcc-arm-none-eabi-4_7-2012q4/bin/../lib/gcc/arm-none-eabi/4.7.3/../../../../arm-none-eabi/lib\libc.a(lib_a-reent.o)
 .debug_frame   0x0000113c       0x3c c:/ti/ccsv5/tools/compiler/gcc-arm-none-eabi-4_7-2012q4/bin/../lib/gcc/arm-none-eabi/4.7.3/../../../../arm-none-eabi/lib\libc.a(lib_a-wbuf.o)
 .debug_frame   0x00001178       0x58 c:/ti/ccsv5/tools/compiler/gcc-arm-none-eabi-4_7-2012q4/bin/../lib/gcc/arm-none-eabi/4.7.3/../../../../arm-none-eabi/lib\libc.a(lib_a-wcrtomb.o)
 .debug_frame   0x000011d0       0x44 c:/ti/ccsv5/tools/compiler/gcc-arm-none-eabi-4_7-2012q4/bin/../lib/gcc/arm-none-eabi/4.7.3/../../../../arm-none-eabi/lib\libc.a(lib_a-wctomb_r.o)
 .debug_frame   0x00001214       0x20 c:/ti/ccsv5/tools/compiler/gcc-arm-none-eabi-4_7-2012q4/bin/../lib/gcc/arm-none-eabi/4.7.3\libgcc.a(_udivsi3.o)
 .debug_frame   0x00001234       0x54 c:/ti/ccsv5/tools/compiler/gcc-arm-none-eabi-4_7-2012q4/bin/../lib/gcc/arm-none-eabi/4.7.3\libgcc.a(bpabi.o)
 .debug_frame   0x00001288       0x38 c:/ti/ccsv5/tools/compiler/gcc-arm-none-eabi-4_7-2012q4/bin/../lib/gcc/arm-none-eabi/4.7.3\libgcc.a(_divdi3.o)
 .debug_frame   0x000012c0       0x38 c:/ti/ccsv5/tools/compiler/gcc-arm-none-eabi-4_7-2012q4/bin/../lib/gcc/arm-none-eabi/4.7.3\libgcc.a(_udivdi3.o)
 .debug_frame   0x000012f8      0x2f8 c:/ti/ccsv5/tools/compiler/gcc-arm-none-eabi-4_7-2012q4/bin/../lib/gcc/arm-none-eabi/4.7.3/../../../../arm-none-eabi/lib\librdimon.a(rdimon-syscalls.o)
 .debug_frame   0x000015f0       0x28 c:/ti/ccsv5/tools/compiler/gcc-arm-none-eabi-4_7-2012q4/bin/../lib/gcc/arm-none-eabi/4.7.3/../../../../arm-none-eabi/lib\librdimon.a(rdimon-_exit.o)
 .debug_frame   0x00001618       0x2c c:/ti/ccsv5/tools/compiler/gcc-arm-none-eabi-4_7-2012q4/bin/../lib/gcc/arm-none-eabi/4.7.3/../../../../arm-none-eabi/lib\librdimon.a(rdimon-_kill.o)
 .debug_frame   0x00001644       0x20 c:/ti/ccsv5/tools/compiler/gcc-arm-none-eabi-4_7-2012q4/bin/../lib/gcc/arm-none-eabi/4.7.3/../../../../arm-none-eabi/lib\libc.a(lib_a-errno.o)

.debug_ranges   0x00000000       0x20
 .debug_ranges  0x00000000       0x20 ./startup_ARMCA8.o
